:020000020000FC
:0200000039C005
:02003C00C6C03C
:040050000C94B0005C
:100070000C94C40000E40EBF0FEF0DBF0E9491036B
:10008000789400911701002379F400911601002360
:1000900051F4009100010023A1F300270093000117
:1000A0000E94F000EECF3DC00E94DF0000911701DA
:1000B000102F0E941C0B009117010117C9F7009324
:1000C00019010E940B0E623319F0F0FE0E94120912
:1000D0000E94E70D0027009334010E945E250091E5
:1000E000170110911901011791F0102F0E941C0B9C
:1000F000009117010117C9F70E940B0E0E94120907
:100100000E94E70D0027009334010E945E25B1E1B3
:10011000A6E3002700931701009319010E94D9005C
:10012000B0CF0E94DF00102F0E941C0B009116011F
:100130000117C9F7009318010E94050E0E945E2561
:100140000091160110911801011701F0D2E1C6E3E8
:10015000002700931601009318010E94D90091CF47
:100160000F930FB70F930091170103950093170199
:100170000091C6000D93623319F0D0FE0E94730304
:100180000F910FBF0F9118950F930FB70F93009119
:100190001601039500931601002311F4D2E1C6E382
:1001A0000091CE0009930E947C030F910FBF0F9125
:1001B00018950F9302E000936F000F9108950F932D
:1001C00000E000936F000F9108950F930FB70F9306
:1001D00000270395009300010F910FBF0F91189511
:1001E0000F930E94E60E0E94D60EA8950E948A10D8
:1001F00080FD14C181FD12C10E94C91082FD69C138
:1002000083FD67C184FD65C185FD63C174FD0E94E6
:10021000351377FD0E94351372FD0E94AC027727DB
:10022000643189F0653191F0623050F06630A8F0A9
:100230006630F1F0673051F0683029F0623311F028
:100240000F91089506C00E94CE0E53C00E94CE0E9C
:100250004DC00E947C010F9108950E94B101D3FE10
:100260000E94DE0E0E94CE0E0F9108950F91089508
:10027000F0FE06C00E94CE0E0E9444010F91089528
:100280000E94BF1A0F910895009109010395043649
:1002900031F500270093090100910A0103950A3006
:1002A00009F100930A01013019F0093089F008952D
:1002B0000E94A508F7E6E0E70E94D30805EE0E9439
:1002C0007C0305EB0E947C030AE40E947C030895F2
:1002D0000E94A508F8E6E0EF0E94D3080895009375
:1002E00009010895002700930A0108953BD10F9159
:1002F000089563D10F91089510910D01112371F1AB
:1003000000910B0103950436F9F4002700930B01CB
:1003100000910C0103950A30E1F4002700930C01D1
:1003200020910E012395211750F0222720930E01D2
:10033000FAE6EAEC0E9485030E94CE0E089520930F
:100340000E010E94CE0E089500930B010E94CE0E66
:10035000089500930C010E94CE0E08950E94CE0EC7
:100360000895009109010395043669F5002700936B
:10037000090100910A010395013061F0023089F012
:100380000330B1F00A30E1F4002700930A01623033
:10039000E8F4089500930A01D1FE11C00E94B4133D
:1003A000089500930A01D1FE0AC00E94C91308955E
:1003B00000930A01D1FE03C00E94D413089508954A
:1003C00000930A010895009309010895D4FE11C015
:1003D000D5FC0BC00E94F90D0E94A008F9E6E0E2EE
:1003E0000E94D3080E94BA0A04C00E94FF0D0E9416
:1003F000C60AD1FE01C00895009134011091350163
:10040000011741F40027009334010E94E10D0E947E
:100410001209089503950093340108950E94290D4F
:10042000062F003011F1063020F1063051F107306F
:1004300061F1083071F1023301F10A3071F10B30D2
:1004400081F10C3091F1043181F0053191F00631E8
:1004500081F1073191F1083161F00B3151F008322F
:10046000A1F10E3170F50F9108950E94621B0F915A
:1004700008950E94631C0F9108950E9402200F911D
:1004800008950E94A51A0F9108950E94421E0F918F
:1004900008950E94501F0F9108950E943B220F91D2
:1004A00008950E94FF220F9108950E94DC230F916E
:1004B00008950E9498200F9108950E9456210F914F
:1004C00008950E945B240F9108950E94F6240F91D5
:1004D0000895062F0030C1F00130D1F00730E1F06F
:1004E0000830F1F00A3061F10B3071F10C3081F11C
:1004F000043151F0053161F00631B1F00731C1F03E
:100500000832D1F00F9108950E94241B0F91089595
:100510000E94021C0F9108950E94E81D0F910895FA
:100520000E94111F0F9108950E946C200F91089551
:100530000E94FE200F9108950E94BC240F910895FF
:100540000E94C2210F9108950E94D0220F91089518
:100550000E94B8230F910895062F002311F40E94E2
:10056000E0090895F1FC0E94080300910101039540
:100570000B3419F000930101089500270093010145
:10058000009102010395023029F0043151F00093EB
:1005900002010895009302010E9453120E94A009D3
:1005A00008950027009302010BE817D6F9E6E2E070
:1005B0000E94D3080E94A0090895F1FC0E9408033C
:1005C0000091010103950B3419F000930101089586
:1005D000002700930101009102010395023029F0E8
:1005E000043151F0009302010895009302010E942A
:1005F00053120E94A00908950027009302010E944F
:1006000053120E94A508F8E6E0EF0E94D30808956F
:1006100000913713039500933713053309F00895BC
:100620000027009337130091361303950093361378
:100630000130B9F0023019F0033069F008950AE58D
:100640000E947C0301E80E947C030EE70E947C0369
:10065000B1E1A6E308950E943909002700933613FB
:1006600008950E947F0E0E948B0EF4FE30C0B3E10D
:10067000A0E403EA0D93009138130D930091391310
:100680000D9300913A130D9300913B130D9305E0E8
:1006900000934E130E94C7160D9300950C93B3E17F
:1006A000A0E40D910E947C030D910E947C030D91AA
:1006B0000E947C030D910E947C030D910E947C039B
:1006C0000D910E947C030C910E947C0308950AE91D
:1006D0000E947C030FEC0E947C0300E30E947C03D9
:1006E000B1E1A6E308951F931091C80015FFFCCF58
:1006F0000093CE001F9108951F931091C00015FF25
:10070000FCCF0093C6001F9108950F930591003010
:1007100011F0F2DFFBCF0DE0EFDF0AE0EDDF0F912C
:1007200008950E94FE0EF894159A129A139A149A3C
:10073000109A119A0027059B006F029B0F600FE330
:1007400004B90AEC0AB9599A5B9A5F9A0E94870821
:100750000E94CD080E947E050E94F4040E94B0050C
:100760000E94C10500270093030100930401009338
:10077000050100930601009301010093020100931B
:1007800007010093090100930A0100930E010093F1
:1007900016010093170100931801009319010093AB
:1007A000340100931C0100930B0100930C0103958D
:1007B00000930D0100931D010FEF00932D01009395
:1007C0002E0100932F0100933001BB24CC24DD24A3
:1007D000EE24FF24AA243324442488277724662483
:1007E000772755240E9449040E9440040E947C0BF4
:1007F0000E9427060E94EA040E9474040E949C043E
:100800000E94D3040E94DB040E943C040E94900DCD
:100810000E943B0E0E94230E0E942F0E0E94410E4A
:100820000E94F30D0E94CF0D0E94DB0D0E94E70D88
:100830000E94170E0E94C9100E94C9100E9415063E
:100840000E9425040E940C0F08950E94CD08662383
:1008500019F40E94DE170895613019F40E94F4170C
:100860000895663028F40E94BD0D0E943418089542
:1008700062330E940A180895B6FC0E946B06089520
:1008800011270E948F0CB02E11E00E948F0CC02EF9
:1008900008950E94BA0C003108F0002700931E0151
:1008A0000E94C40C063008F0002700931F010E942C
:1008B000CE0C083008F00027009320010E94D80CCD
:1008C000093008F00027009321010E94E20C053056
:1008D00008F00027009322010E94EC0C073008F07A
:1008E00000270093230108950E94A60C0B3018F0F6
:1008F00000270E94A10C002E0B2D04FF07C0F4E777
:10090000E6E1002DE00F48F4F39507C0F4E7E2E2DA
:10091000002DE00F10F4F39500C00491202E0E94EA
:10092000B00C102E0F3F19F00395021520F0002790
:100930000E944A12112408950E949C0C602F0630D8
:1009400038F0023329F000270E944A120E94BF0C9F
:1009500000932601602F0023F9F0013029F40E9452
:10096000540C0093330118C0162F0E942F0C0093D3
:100970003101162F0E94450C00933301162F0E945F
:100980007B0C00933201162F0E94650C00931A0114
:100990000E94F60C00931B010895DACF0E947B0C95
:1009A00000933201D5CF00913301043008F00027C5
:1009B0000093330108950E940A0D002329F00B30A3
:1009C00018F400933501089505E00E944A1200933F
:1009D000350108950E94000D002311F0053008F044
:1009E00001E000930801089502990895059908957A
:1009F0000E942C0B0E94A008F9E6E8E90E94D308A7
:100A00000E94A508F9E6EAEA0E94D3080E942C0B8E
:100A10000E942C0B0E942C0B0E942C0B0E94A00801
:100A2000F9E6ECEB0E94D3080E94A508F9E6EEEC8B
:100A30000E94D3080E942C0B0E942C0B0E942C0BAE
:100A40000E942C0B0E942C0B0E942C0B029947C079
:100A5000059945C00E94CD080E94A008F9E6E0EE85
:100A60000E94D3080E94A508F0E0E0E011270E9450
:100A7000C1050E94160F00270E944A123196139555
:100A8000143021F411270EE20E94DB08F999FECF01
:100A90000E945C0B0E945C0B0E945C0B0E945C0B32
:100AA0000E945C0BF03039F7EF3329F70EE20E9419
:100AB000DB08002701600D7F0460077F0061006292
:100AC000006411270E94850C002711E00E94850C0C
:100AD00000270E7F0D7F12E00E94850C0EC00E9441
:100AE000A008FAE6E4E00E94D3080E94A508FAE60E
:100AF000E6E10E94D3080E94160FFFCF0E94140D5A
:100B0000023409F408950E94A008FAE6ECE40E9479
:100B1000D3080E94A508FAE6E8EB0E94D308F0E0AB
:100B2000E0E002E40E940F0D0E945C0B0E945C0B4F
:100B30000E94160F002701600D7F0460077F00618F
:100B40000062006411270E94850C002711E00E94BA
:100B5000850C00270E7F0D7F12E00E94850CCDCF03
:100B6000029908950E942C0B0E94A008F0E6E8E983
:100B70000E94D3080E94A508F0E6E8E90E94D30885
:100B8000FFCF059908950E942C0B0E94A0080E9497
:100B9000A008F7E6E2E80E94D3080E94A5080E9498
:100BA0005C0BF8E6E0EF0E94D3080E94A5080E94C3
:100BB0005C0BF9E6E2E00E94D3085527539540E329
:100BC000052F040F0E94DB08059B0BC0029B01C090
:100BD000FBCF029BFECF052F009308010E94FB0C68
:100BE00008950E945C0B059BFCCF0E945C0B059B4B
:100BF000FCCF0E94A5080E945C0BF8E6E0EF0E9483
:100C0000D3080E94A5080E945C0BF9E6E2E00E946E
:100C1000D3085395553039F040E3052F040F0E9457
:100C2000DB080C94E40550E0E0CF00913201053080
:100C300018F001E0009332010E949D0E002708E1A8
:100C40000093C100002708E10093C90008950FEF49
:100C500013E8009385001093840000E01CE70093E4
:100C60008900109388000BE0009381000E94D90056
:100C70000895059BFECF0E94A008F0E6E8E90E94D7
:100C8000D3080E94A508F0E6E8E90E94D308FFCF48
:100C90000E94A008F7E6E4E90E94D3080E94A50894
:100CA000F7E6E6EA0E94D3080E94660608950E94CD
:100CB000A008F7E6E8EB0E94D3080E94A508F7E633
:100CC000EAEC0E94D3080E94660608950E942C0B4D
:100CD0000E942C0B08950E944806029BA1C0059B10
:100CE000A6C00E945706029B9BC0059BA0C066231E
:100CF00031F06130E9F0663008F008953EC00E949E
:100D0000C60A029B8DC0059B92C00E94F407029BFD
:100D100087C0059B8CC00E940C08029B81C0059B6C
:100D200086C00E943D08029B7BC0059B80C0089541
:100D30000E942407029B74C0059B79C00E943B0758
:100D4000029B6EC0059B73C00E94F407029B68C0A3
:100D5000059B6DC00E940C08029B62C0059B67C08A
:100D60000E942408029B5CC0059B61C00E943D0854
:100D7000029B56C0059B5BC008950E942407029BFE
:100D80004FC0059B54C00E943B07029B49C0059B76
:100D90004EC00E945307029B43C0059B48C00E945F
:100DA0006B07029B3DC0059B42C00E948507029BCA
:100DB00037C0059B3CC00E94BC07029B31C0059B0D
:100DC00036C00E94F407029B2BC0059B30C00E94D6
:100DD0000C08029B25C0059B2AC00E942408029B88
:100DE0001FC0059B24C00E943D08029B19C0059BA3
:100DF0001EC00E945508029B13C0059B18C000919D
:100E00003101002361F0023051F0033041F008302D
:100E100031F00E946E08029B03C0059B08C0089534
:100E20000E94CD080E945C0B02990895FBCF0E949E
:100E3000CD080E945C0B05990895FBCF002319F0A3
:100E40000A957296FBCF08950E94CD080E94A008D3
:100E5000F1E6ECED00270E941E070E94D3080E94D5
:100E6000A508F3E6EEE0062F0E941E070E94D308B5
:100E70000E94660608950E94CD080E94A008F1E62F
:100E8000ECED01E00E941E070E94D3080E94A50815
:100E9000F3E6E0EB009133010E941E070E94D308A5
:100EA0000E94660608950E94CD080E94A008F1E6FF
:100EB000ECED02E00E941E070E94D3080E94A508E4
:100EC000F4E6E2E5009131010E941E070E94D3087A
:100ED0000E94660608950E94CD080E94A008F1E6CF
:100EE000ECED03E00E941E070E94D3080E94A508B3
:100EF0000E947B0CF5E6E6E0009132010E941E079D
:100F00000E94D3080E9466060895009131010130C5
:100F100019F0083009F008950E94CD080E94A00839
:100F2000F9E6E6E80E94D30800911A010E94D50A6A
:100F300000911B010E94F10A0E9466060091310196
:100F4000013019F0083009F008950E94CD080E9480
:100F5000A008F1E6ECED05E00E941E070E94D30810
:100F600005EC0E94ED08F6E6EAEDB0FE38960E9428
:100F7000D3080E946606089500913101002329F0EC
:100F8000023019F0033009F008950E94CD080E9444
:100F9000A008F1E6ECED06E00E941E070E94D308CF
:100FA00005EC0E94ED08F6E6EAED7096B1FE389683
:100FB0000E94D3080E9466060E94CD080E94A008E5
:100FC000F1E6ECED07E00E941E070E94D30805EC55
:100FD0000E94ED08F6E6EAED7096C1FE38960E9492
:100FE000D3080E94660608950E94CD080E94A008BA
:100FF000F1E6ECED08E00E941E070E94D30805EC24
:101000000E94ED08F6E6EAEDB096B2FE38960E9430
:10101000D3080E94660608950E94CD080E94A00889
:10102000F1E6ECED09E00E941E070E94D30805ECF2
:101030000E94ED08F6E6EAEDF096B3FC38960E94C1
:10104000D3080E94660608950E94CD080E94A00859
:10105000F1E6ECED0AE00E941E070E94D30805ECC1
:101060000E94ED08F6E6EAEDF0967096B4FE38962A
:101070000E94D3080E94660608950E94CD080E942F
:10108000A008F1E6ECED0BE00E941E070E94D308D9
:1010900005EC0E94ED08F6E6EAED7096B5FE38968E
:1010A0000E94D3080E94660608950E94CD080E94FF
:1010B000A008F1E6ECED0EE00E941E070E94D308A6
:1010C00005EC0E94ED080E94A508F7E6EAE30E94FD
:1010D000D3080E94DE240E94660608950E94CD086F
:1010E0000E94A008F1E6ECED0FE00E941E070E94AE
:1010F000D30805EC0E94ED08F6E6EAEDF096B0960E
:10110000C0FE38960E94D3080E9466060895002704
:10111000006105B92C9A299A289A6FD06ED06DD0AB
:1011200028986BD02998F1E1E8E30591003019F097
:1011300054D0D2D2FACF08952808061701020C0025
:101140000F9300E84AD00F9108950F9300EC45D01B
:101150000F9108950F9300EC40D00F9108950F93D5
:1011600002EC3BD00F9108950F930DEC36D00F9108
:1011700008950F930CEC31D00F9108950F9308EC64
:101180002CD00F9108950F9307EC27D00F9108955D
:101190000F930DEC22D00F9108950F9301E01DD015
:1011A0009BD20F9108950F930591003011F003D059
:1011B000FBCF0F9108950F930F93007F029500626C
:1011C000006105B91AD00F910295007F0295006267
:1011D000006105B912D00F9108950F930F93007F0E
:1011E0000295006105B909D00F910295007F029523
:1011F000006105B902D00F9108952C9A03D02C9864
:101200003BD2089508950F930091330100E8F1FE59
:1012100005E8E3DF10E3009133010395010FCBDF15
:101220000F9108950F9307E8D8DF663031F06730EB
:1012300048F4D1FC04C003E4BEDF0F91089503E538
:10124000BADFFBCF00E2B7DFF8CF0F9309E8C5DFC5
:10125000E2FC06C0E3FC06C0E4FC06C000E205C0F8
:101260000DE303C00BE201C00DE20E94DB080F9109
:10127000089502E8B2DFF3FC1EC0F2FE3AC000910E
:101280003F1399DF00913E1396DF0EE294DF0EE2EA
:1012900000913D1390DF00913C138DDF0DE00AE0DB
:1012A00000E289DF08E587DF00914F1384DF002724
:1012B00000935613089509E30E94DB080E94DB089F
:1012C0000EE20E94DB0809E30E94DB080E94DB08B3
:1012D00000E20E94DB0808E50E94DB0800914F1342
:1012E0000E94DB08002700935613F4FE0E94910E23
:1012F0000895009156130395053031F0009356136D
:10130000F4FE0E94910E08950DE20E94DB080E94F7
:10131000DB080EE20E94DB080DE20E94DB080E945F
:10132000DB0800E20E94DB0800E20E94DB080E946A
:10133000DB08002700935613F4FE0E94910E0895D7
:101340000F930CD000E237DF36DF35DF39D000E213
:1013500032DF31DF30DF19D00F910895FBDE032D2E
:1013600007FD00584AD0B2FE0DC0032D132D009585
:10137000103828F4003808F0005812D0089500689A
:101380000FD00895032D0CD008950B2D03FF02C03C
:10139000F0DE01C0E9DE042D5ED0042D09D00895F1
:1013A0000F93BED10F9114E1202FCED1E4D1089537
:1013B0000F93B6D10F9115E1202FC6D1DCD108953E
:1013C000DDDE032D07FF03C008E4F5DE02C004E5FF
:1013D000F2DE00E5F0DEB2FE0DC0032D132D009508
:1013E000103828F4003808F00058DADF0895006853
:1013F000D7DF0895032DD4DF089544275527F3E759
:10140000E8EE032D07FD005818E0079528F0329606
:101410001A951123D1F705C025913591420F531F1D
:10142000F7CF042F152F0E94FD1510E3042F0F7026
:10143000010FC1DE032F007F0295010FBCDE0EE21B
:10144000BADE032F0F70010FB6DE022F007F029568
:10145000010FB1DE0895442755270B2D03FF19F026
:10146000F4E7E6E002C0F3E7E6EF042D18E00795A5
:1014700028F032961A951123D1F705C025913591A0
:10148000420F531FF7CF042F152F0E94FD1510E3B5
:10149000032F0F70010F0E94DB08022F007F0295BF
:1014A000010F89DE022F0F70010F85DE0B2D03FF68
:1014B00002C000E380DE089511270E94FD1510E3AD
:1014C000032F0F70002311F400E301C0010F73DE3E
:1014D00010E3022F007F0295010F6DDE022F0F70C7
:1014E000010F69DE08951F930F930E94FD150BE80D
:1014F00074DE10E3042F0F70002311F400E201C02A
:10150000010F59DE10E3032F007F0295010F53DE18
:10151000032F0F70010F4FDE10E3022F007F0295A3
:10152000010F49DE022F0F70010F45DE1F910F9151
:1015300008952CD068DE623020F0673010F40C94EF
:10154000A70A07E84ADE00E236DE0C94A80A6ADE43
:101550007CDEA9D76BD7B2D6E00FF11F93D7402E10
:1015600065D7C9D6E00FF11F8DD7302EE9DE0E9476
:10157000250D089548DE56DE68DE0BE82EDEF9E61E
:10158000E6E211DEDDDE0E94290D08950E94A0082A
:10159000F9E6E8E10E94D308062F1FE2010F0E943E
:1015A000DB0800E20E94DB08089500911A010F9306
:1015B000007F02950A3010F410E302C00A5011E4D3
:1015C000100F02EC0ADE012FF6DD0F910F700A30CA
:1015D00010F410E302C00A5011E4100F012FEBDDEC
:1015E000089500911B010F93007F02950A3010F4BB
:1015F00010E302C00A5011E4100F0CECEEDD012FD5
:10160000DADD0F910F700A3010F410E302C00A50B7
:1016100011E4100F012FCFDD089502ECDEDD009103
:101620001C0111E3010FC7DD0DECD7DD00911D0199
:1016300011E3010FC0DD08950F931F932F932EE048
:1016400010E10DEE0150F1F71150D9F72150C1F71B
:101650002F911F910F9108951F932F933F933BE676
:1016600022EB15E41150F1F72150D9F73150C1F7B1
:101670003F912F911F9108951F932F933F9331E036
:101680002FE311E01150F1F72150D9F73150C1F794
:101690003F912F911F9108950F931F932F9321E056
:1016A0001DED05E00150F1F71150D9F72150C1F7B8
:1016B0002F911F910F9108951F932F933F9336E021
:1016C0002CE314E21150F1F72150D9F73150C1F752
:1016D0003F912F911F9108950F931F932F932AE00D
:1016E00017E40EE00150F1F71150D9F72150C1F77E
:1016F0002F911F910F9108950091B9000C7F006008
:101700000093B90000E20093B8000AD010E020E096
:101710001BD031D005D011E020E016D02CD0089598
:1017200004EA0093BC0004EA0093BC002CD043D030
:1017300004E00093BC0000E40093BB0004E80093C5
:10174000BC0021D03FD0089504E00093BC00012FDD
:101750000093BB0004E80093BC0015D039D004E02E
:101760000093BC00022F0093BB0004E80093BC0070
:101770000AD02ED0089504E90093BC000091BC006B
:101780000071E1F708951F932F933F9311272227AC
:1017900033270091BC0007FF04C03F912F911F9198
:1017A000089513951123A9F72395222391F73395D3
:1017B000393179F713C060DF0091B900087F083034
:1017C000D1F408950091B900087F083109F5089512
:1017D0000091B900087F083241F508950E94A008E1
:1017E000F7E6E6EA0E94D3080E94A508F7E6ECEDCA
:1017F0000E94D30827C00E94A008F7E6E6EA0E94EC
:10180000D3080E94A508F7E6EEEE0E94D3081AC09E
:101810000E94A008F7E6E6EA0E94D3080E94A50805
:10182000F8E6E0E00E94D3080DC00E94A008F7E6A9
:10183000E6EA0E94D3080E94A508F8E6E2E10E94C9
:10184000D30800C0FFCF0F9300271A951A95F0E038
:10185000E9E0E10FF01F0F910E944A12089500275E
:101860001A951A95F0E0E9E0E10FF01F0E9442128C
:1018700008950F9300271A951A95F0E0EDE0E10F17
:10188000F01F0F910E944A12089500271A951A9589
:10189000F0E0EDE0E10FF01F0E9442120895F0E049
:1018A000E1E10E944A120895F0E0E1E10E94421253
:1018B00008950F9300271A951A95F0E0E6E1E10FDD
:1018C000F01F0F910E944A12089500271A951A9549
:1018D000F0E0E6E1E10FF01F0E94421208950F933D
:1018E00000271A951A95F0E0E2E1E10FF01F0F9141
:1018F0000E944A12089500271A951A95F0E0E2E135
:10190000E10FF01F0E94421208950F930027F0E0AC
:10191000EBE1E10FF01F0F910E944A12089500279A
:10192000F0E0EBE1E10FF01F0E9442120895F0E0B9
:10193000E0E00E944A120895F0E0E0E00E944212C6
:101940000895F0E0E1E00E944A120895F0E0E1E03D
:101950000E9442120895F0E0E2E00E944A120895C7
:10196000F0E0E2E00E9442120895F0E0E3E00E941D
:101970004A120895F0E0E3E00E9442120895F0E078
:10198000E4E00E944A120895F0E0E4E00E9442126E
:101990000895F0E0E5E00E944A120895F0E0E5E0E5
:1019A0000E9442120895F0E0E6E00E944A12089573
:1019B000F0E0E6E00E9442120895F0E0E7E00E94C5
:1019C0004A120895F0E0E7E00E9442120895F0E024
:1019D000E8E00E944A120895F0E0E8E00E94421216
:1019E0000895F0E0EAE10E944A120895F0E0EAE189
:1019F0000E9442120895F0E0E8E20E944A1208951F
:101A0000F0E0E8E20E9442120895F0E0E9E20E946C
:101A10004A120895F0E0E9E20E9442120895F0E0CF
:101A2000EAE20E944A120895F0E0EAE20E944212BD
:101A3000089500913101013021F0083011F05E98D5
:101A40000895B0FEFCCF5E9A0895B5FE01C05F9880
:101A50000895B5FE01C05F9A089574FF04C00B2D70
:101A600001600C94350D0B2D0E7FB02E11270E94B6
:101A7000850C0E94190D089574FF04C00B2D02609F
:101A80000C94440D0B2D0D7FB02E11270E94850C58
:101A9000089574FF04C00B2D04600C94510D0B2DA0
:101AA0000B7FB02E11270E94850C089574FF04C08F
:101AB0000B2D077F0C945E0D0B2D0860B02E1127A7
:101AC0000E94850C089574FF04C00B2D00610C94D6
:101AD0006B0D0B2D0F7EB02E11270E94850C0895E3
:101AE00074FF04C00B2D00620C94780D0B2D0F7D3C
:101AF000B02E11270E94850C089574FF04C00B2D91
:101B000000640C94850D0B2D0F7BB02E11270E94C5
:101B1000850C08950F930E2D0160E02E0F9108950E
:101B20000F930E2D0E7FE02E0F91089574FF04C0C9
:101B30000C2D01600C949E0D0C2D0E7FC02E11E01B
:101B40000E94850C00913101002349F0023039F0E8
:101B5000033029F0083019F00E2D0E7FE02E089585
:101B600074FF04C00C2D02600C94B80D0C2D0D7F79
:101B7000C02E11E00E94850C08950F930D2D006179
:101B8000D02E0F9108950F930D2D0F7ED02E0F9113
:101B900008950F930D2D0064D02E0F9108950F938B
:101BA0000D2D0F7BD02E0F9108950F930D2D0068F2
:101BB000D02E0F9108950F930D2D0F77D02E0F91EA
:101BC00008950F930D2D0260D02E0F9108950F935D
:101BD0000D2D0D7FD02E0F9108950F930D2D0160C7
:101BE000D02E0F9108950F930D2D0E7FD02E0F91B3
:101BF00008950F930D2D0062D02E0F9108950F932D
:101C00000D2D0F7DD02E0F9108950F930D2D046093
:101C1000D02E0F9108950F930D2D0B7FD02E0F9185
:101C200008950F930D2D0860D02E0F9108950F93F6
:101C30000D2D077FD02E0F9108950F930E2D00626A
:101C4000E02E0F9108950F930E2D0F7DE02E0F9132
:101C500008950F930E2D0064E02E0F9108950F93B9
:101C60000E2D0F7BE02E0F9108950F930E2D026025
:101C7000E02E0F9108950F930E2D0D7FE02E0F9102
:101C800008950F930E2D0B7F077F0F7EE02E0F918F
:101C900008950F930E2D0460077F0F7EE02E0F91A5
:101CA00008950F930E2D0B7F08600F7EE02E0F918D
:101CB00008950F930E2D0B7F077F0061E02E0F918B
:101CC00008950F930F2D0160F02E0F9108950F933B
:101CD0000F2D0E7FF02E0F9108950F930F2D0260A0
:101CE000F02E0F9108950F930F2D0D7FF02E0F9171
:101CF00008950F930F2D0460F02E0F9108950F9308
:101D00000F2D0B7FF02E0F9108950F930F2D08606C
:101D1000F02E0F9108950F930F2D077FF02E0F9146
:101D200008950F930F2D0061F02E0F9108950F93DA
:101D30000F2D0F7EF02E0F91089500913201002398
:101D400049F0013059F0023069F0033079F0043085
:101D500089F004C050E047E626E00FC050E043E3BE
:101D600026E00BC050E049E126E007C050E04CE01F
:101D700026E003C050E047E62EE05093C5004093B4
:101D8000C4002093C2005093CD004093CC00209318
:101D9000CA00B1E1A6E3D2E1C6E308950F93009132
:101DA000C10000680093C1000F9108950F93009146
:101DB000C1000F770093C1000F9108950F93009118
:101DC000C90000680093C9000F9108950F93009116
:101DD000C9000F770093C9000F9108950F930091E8
:101DE000C90000610093C9000F9108950F930091FD
:101DF000C9000F7E0093C9000F910895F894A8952B
:101E000004B7077F04BF0091600008610093600081
:101E100000E0009360000895009160000861009365
:101E2000600009E200936000A895089500916000A9
:101E30000861009360000EE000936000A89508958B
:101E40000E94ED0D0E94FE0E00E000936F000E94C4
:101E5000A008FAE6EEE50E94D3080E94A508FAE67B
:101E6000E2E80E94D3080FEF602F0E94DE0E0E946E
:101E7000CE0E7894002700931701B1E1A6E30091FC
:101E800017010023E1F3B1E1A6E30C910334C1F69D
:101E9000F0E0E0E0319741E001E00E947C03042F94
:101EA0000E947C0300950E947C0322273327209305
:101EB0000F013093100150E831960E9442120E94A7
:101EC0007C03FBD65A955523B9F7002700931701D9
:101ED000B1E1A6E3009110010E947C0300910F0183
:101EE0000E947C03009117010023E1F3B1E1A6E316
:101EF0000C910630B1F0053121F4FF97FF9732972E
:101F0000CBCF0E94A008FAE6E4E90E94D3080E9421
:101F1000A508FAE6E8EB0E94D3080E94160F0C947D
:101F20007D054395413261F7002700931701B1E128
:101F3000A6E304E00E947C03009117010023E1F373
:101F4000B1E1A6E30C910630E1F6002700931701FA
:101F5000B1E1A6E307E10E947C030E940C0F0E94FE
:101F6000F30D02E000936F0008950E94ED0D0E94B2
:101F7000FE0E00E000936F00882499240E94A008C0
:101F8000FAE6E0E70E94D3080E94A508FAE6E2E834
:101F90000E94D3080FEF602F0E94DE0E0E94CE0E2B
:101FA0007894F1E0E6E33197002700931701B1E15F
:101FB000A6E333274427552703E40E947C030091BE
:101FC0001701002371F433953323C9F74395442354
:101FD000B1F753955D3299F75527E6CF50C04FC002
:101FE0005EC0009117010023E1F3332744275527F2
:101FF00033953323E9F743954423D1F7539555306F
:10200000B9F75527B1E1A6E30C910430B9F100917D
:102010001701053819F7B1E1A6E30D910130F9F682
:102020000D911D91010F0F3F51F5002700931001F5
:1020300000930F0150E80D9140D65A955523D9F7DA
:102040000D911D912091100130910F01021713077E
:1020500039F6B1E1A6E3139650E80D91319600836D
:102060000E9478105A955523C1F700270093170155
:10207000B1E1A6E306E00E947C03B3CF19C00E9441
:10208000A008FAE6E4E90E94D3080E94A508FAE64F
:10209000E8EB0E94D3080E94160F0C947D050027E0
:1020A00000931701B1E1A6E305E10E947C0399CFFB
:1020B00006E00E947C0306E00E947C0306E00E948A
:1020C0007C038820E1F6092D0031C9F60E94A008A2
:1020D000FAE6E6EA0E94D3080E94A508FAE6E8EBD1
:1020E0000E94D3080E94F30D02E000936F00089550
:1020F0001F930F93112701E0800E911E092D0031CF
:1021000031F4082D023018F00F911F91B8CF0F91C4
:102110001F9108958827059B0C949B10029B0C949B
:10212000AE10002700930301009304010093050102
:102130000093060108950160802F0091030103952B
:102140000B3449F400270093030100910401039527
:102150000093040108950093030108950260802F05
:102160000091050103950B3449F400270093050104
:10217000009106010395009306010895009305015F
:1021800008950002010001000002020000010001A8
:10219000020000B10370071581F10F93172D110F85
:1021A000110F012BE2E8F1E22227E00FF21F049168
:1021B000013089F40091070103955091080105173A
:1021C00019F00093070106C0002700930701082FAC
:1021D0000061802F10C00091070103955091080104
:1021E000051719F00093070106C0002700930701A7
:1021F000082F0062802F0F91702E00B10871069594
:1022000006950695061581F10F93162D110F110FE6
:10221000012BE2E8F1E22227E00FF21F04910130E6
:1022200089F400910701039550910801051719F0F1
:102230000093070106C0002700930701082F0460E0
:10224000802F10C0009107010395509108010517D8
:1022500019F00093070106C0002700930701082F1B
:102260000860802F0F91602E0895B4FC03C0F4E73E
:10227000E2E202C0F4E7E6E1002DE00F08F4F39596
:102280000491202E0027F0E0EDE1E00D08F4F39535
:102290000E94421208950E9416120E945E11E00FE1
:1022A000F11F042D0E944A120E9416120E947B11F7
:1022B000E00FF11F032D0E944A1208950F93009121
:1022C0003301002341F0013051F0023061F003305E
:1022D00071F000E0DFD0F2E0ECE20F910895F6E05B
:1022E000E4E10F910895F9E0ECEF0F910895FDE01E
:1022F000E4EE0F9108950F9300913301002341F014
:10230000013051F0023061F0033071F000E0C2D0D2
:10231000F0E0E8E30F910895F4E0E0E20F91089512
:10232000F8E0E8E00F910895FBE0E0EF0F910895E9
:10233000B4FC03C0FCE6E8E502C0FCE6E8E2059177
:102340001591259135911F3FD9F04017510720F085
:102350002417350708F001C0F2CFB4FC03C0F0E742
:10236000ECE202C0FCE6E8E80027009327010093B6
:1023700028010591159104171507A1F11F3F21F4BC
:102380000FEF002E102E08950417150768F4332759
:1023900021E01091270100912801020F131F1093D3
:1023A000270100932801E5CF349725913591041B2F
:1023B000150B4F935F93421B530B242F352F5F91C7
:1023C0004F912017330708F00DC0332721E01091FB
:1023D000270100912801021B130B10932701009382
:1023E000280100C0002700241124B4FC03C0F4E736
:1023F000E2E202C0F4E7E6E105910395112750916E
:102400002701151730F040912801401710F4142EC1
:10241000089540912801509127012227401B510B1C
:1024200040932801509327010394E6CF5F934F9385
:102430003F932F931127222733274427002D502D18
:10244000B4FC03C0F4E7E2E202C0F4E7E6E10023F3
:1024500039F005910395300F411F23952517C9F7D2
:10246000142F032F010D08F413952F913F914F91D5
:102470005F910895F999FECFB2BDA1BDF89A00B55C
:10248000A8950895F999FECFF2BDE1BDF89A00B57F
:10249000A8950895F999FECFF2BDE1BD00BDFA9A65
:1024A000F99AA89508950F931F932F933F934F93F5
:1024B0005F9311272227332744270FEF001509F4D4
:1024C0004DC0002D502DB4FC03C0F4E7E2E202C081
:1024D000F4E7E6E1002339F005910395300F411F41
:1024E00023952517C9F7B4FC03C0F0E7ECE202C05E
:1024F000FCE6E8E80E2F1F2F142F032FE30FF41F25
:10250000E30FF41F012D1127E00FF11FE00FF11F62
:10251000059114910F931F932F933F934F935F93C4
:102520000F921F922F923F924F92512F402F0E9455
:102530009C15009338131093391320933A1330935A
:102540003B134F903F902F901F900F905F914F91B2
:102550003F912F911F910F910E94730A5F914F91AC
:102560003F912F911F910F91089500911C0100231D
:1025700019F4B0E0A8E30CC0013019F4B4E0A0E213
:1025800007C0023019F4B8E0A8E002C0BBE0A0EF39
:1025900000911D01002319F4F0E0E8E30CC00130C4
:1025A00019F4F4E0E0E207C0023019F4F8E0E8E0E2
:1025B00002C0FBE0E0EF112722270E943A120E949E
:1025C0004A12119631961395103029F0143FA9F74D
:1025D000222399F308952395F0CF00911C01002345
:1025E00019F4B2E0ACE20CC0013019F4B6E0A4E199
:1025F00007C0023019F4B9E0ACEF02C0BDE0A4EEB0
:1026000000911D01002319F4F2E0ECE20CC001304E
:1026100019F4F6E0E4E107C0023019F4F9E0E4EE61
:1026200002C0FDE0E4EE112722270E943A120E9428
:102630004A12119631961395112329F0143FA9F7E8
:10264000222399F308952395F0CFF894F0E0E8E37E
:1026500000270E944A120E9442120023C9F73196B5
:10266000F031B1F7E030A1F70895062F002379F19A
:10267000063078F1073079F1083079F10A30D1F17C
:102680000B30D1F10C30D1F10431D1F10531D1F160
:102690000631D1F10731D1F10831E1F10F31F9F013
:1026A0000032F1F00132E9F00232E1F00332D9F008
:1026B0000432D1F00532C9F00632C1F00732B9F068
:1026C0000832B1F00932A9F0023311F108950C94E7
:1026D000721A0C94781A0C94D01A0C94031B00C430
:1026E00002C404C406C408C40AC40CC40EC410C482
:1026F00012C419C40C94EA160C94A1180C94E41991
:102700000C944E1A0C94591A0C949A170C94C419E0
:102710000C941E1BE0FC11C00E948A0D009129013F
:1027200000932B0100912A0100932C0100922E01AD
:10273000109230010E94BF1708950E94900D0E94D0
:10274000BF1708950E94A008F9E6E6E80E94D308A2
:102750000E94A508F8E6E0EF0E94D3080E94D50A7F
:102760000E94F10A66E1089500913101002319F1F8
:10277000013019F10230F9F00330E9F0043031F1A1
:10278000053009F1063001F10730F9F00830C1F0E9
:10279000089500913101002379F0023069F003308F
:1027A00071F0083071F0089500913101033031F07B
:1027B000083041F008950BC016C0A6C02CC01FC041
:1027C00036C059C07EC0D2C0E1C0F9C0C0C009E463
:1027D0000E94730306E40E9473030BE30E947303D9
:1027E0000E94EF14089506E40E94730302E40E941D
:1027F00073030BE30E9473030E94EF1408950FE428
:102800000E94730309E40E9473030BE30E947303A5
:102810000E94EF14089506E40E94730304E50E94E9
:1028200073030BE30E9473030E94EF1408950E9448
:10283000F60E0E94110E0EEF0E9473030EEF0E941F
:10284000730300911A010E94730300911B010E94FF
:10285000730305E20E94730300E00E9473030DEF0F
:102860000E9473030E946C0B0E94EE0E0E94170ED2
:102870000E94EF1408950E94110E0E94F60E0E940D
:10288000E60E0EEF0E9473030EEF0E947303009199
:102890001A010E94730300911B010E94730305E259
:1028A0000E94730301E00E9473030DEF0E94730303
:1028B0000E946C0B0E94EE0E0E94170E0E94EF14F5
:1028C00008950E94110E0E94F60E0E94E60E0EEF71
:1028D0000E9473030EEF0E94730300911A010E947D
:1028E000730300911B010E9473030FE00E947303A6
:1028F0000DEF0E9473030E946C0B0E94EE0E0E946B
:10290000170E0E94EF1408950E94110E0E94F60EF9
:102910000E94E60E0EEF0E9473030EEF0E947303F7
:1029200000911A010E94730300911B010E9473031E
:1029300003E00E9473030DEF0E9473030E946C0B6F
:102940000E94EE0E0E94170E0E94EF1408950027B9
:102950000E9473030E9473030E9473030E94730317
:1029600003E00E9473030E94EF14089500270E9461
:1029700073030E9473030E94730302E00E947303B7
:1029800000E10E9473030E94EF14089500270E9443
:1029900073030E9473030E9473030E9473030E94D7
:1029A00073030E9473030E9473030E9473030E94C7
:1029B000730303E00E9473030E94EF14089500273D
:1029C0000E9473030E9473030E94730303E00E943A
:1029D000730300E10E9473030E94EF140895052D14
:1029E0000A3011F0539408950E94BD0D0E94DB2619
:1029F00008950F931F932F933F934F935F936F937C
:102A00007F938F93F1E1E6E33396219131914191E8
:102A100050810E9421160E94A50800E20E94DB0856
:102A200003E50E94DB080FE20E94DB080EE40E942F
:102A3000DB0800E20E94DB0810E3082F15D0072F07
:102A400013D0062F11D0052F0FD0042F0DD000E288
:102A50000E94DB088F917F916F915F914F913F9121
:102A60002F911F910F9108950F9302950F70010FF1
:102A70000E94DB080F910F70010F0E94DB08089580
:102A8000889408E1302E0027112722273327001CC5
:102A9000111C221C001F111F221F331F3A9409F41E
:102AA0000895402F0BD0042F412F08D0142F422F10
:102AB00005D0242F432F02D0342FE9CF542F5D5F50
:102AC00053FD452F542F505D57FD452F08950F920C
:102AD00016E0012E55274427E8940A9491F01191AD
:102AE0001032D9F31033C9F3105370F01A3060F478
:102AF0000FD056F0410F119110F4539529F00A941C
:102B000099F735970F90089531970F90689408952D
:102B10003F932F93352F242F440F551F48F0440F18
:102B2000551F30F0420F531F18F0440F551F08F483
:102B300068942F913F9108950F921F922F926F9357
:102B40007F9373E068EE2224759F9001649F80015B
:102B5000749F100D211D321D569F100D211D321D19
:102B60007F916F912F901F900F9008950F921F9259
:102B70002F923F922AE0429F202C312C529F212DF0
:102B8000300C08F42395532D422D3F902F901F9029
:102B90000F9008950F921F922F923F924F925F9243
:102BA0006F9210915113109F202C312C10915213C1
:102BB000109F412C300C08F4439410915313109F34
:102BC000512C400C08F4539410915413109F612C15
:102BD000500C08F463942092511330925213409297
:102BE000531350925413609255136F905F904F900F
:102BF0003F902F901F900F9008950F931F935F9316
:102C00006F93AF93BF93222733274427BB2750E10D
:102C1000A5E16E916D5F63FD6C936C91605D67FDE6
:102C20006C93A231B1F7000F111F221F331F441FF5
:102C30005A9571F7BF91AF916F915F911F910F916D
:102C400008950E94471677278EEF4D5C43FF43504F
:102C500047FF40535D5C53FF535057FF50536D5C2B
:102C600063FF635067FF6053220F331F441F551FDC
:102C7000661F771F881F4AF3111FF0F47D5C73FFF6
:102C8000735077FF70538D5F83FF8350DECF042F27
:102C9000152F6FEF639500511742E0F75FE9505130
:102CA00008511C4FE0F3539504561040E0F740EAFA
:102CB0004051065FE8F3400F08954F935F932091D2
:102CC000100130910F012027522F52955F70252758
:102CD000522F5295507F3527522F5295452F507FB6
:102CE0004F70550F441F2527342720930F01309331
:102CF00010015F914F91089550E2EE27FF27110FC9
:102D0000221F331F441FEE1FFF1F18F0EC17FD0793
:102D100018F01395EC1BFD0B5A9589F70895FF9356
:102D2000EF93BF93AF931F93B1E1A6E313962FE008
:102D30000CC0FF93EF93BF93AF931F93B1E1A6E352
:102D4000209117012A952A952A95F4E7EEE211279A
:102D50000D91E00FF11F14910D910127F4E7EEE2C0
:102D60001127E00FF11F14912A952223A9F70D9145
:102D7000011731F410950C91011711F4002701C0CF
:102D800001E01F91AF91BF91EF91FF910895FF93E3
:102D9000EF93BF93AF931F93B3E1A0E420914E1341
:102DA0002A95F4E7EEE211270D91E00FF11F14913F
:102DB0000D910127F4E7EEE21127E00FF11F1491C6
:102DC0002A952223A9F7012F1F91AF91BF91EF916F
:102DD000FF91089575FFC2C000911E010E94B50CBD
:102DE000003069F0013059F0023049F0033039F019
:102DF000043031F00D3031F0003118F008959DC1EC
:102E0000A1CC46C00E9448060E9457066091260148
:102E1000662329F0613061F06630B8F0B0C00E94DE
:102E2000C60A0E94F4070E940C080E943D08A7C031
:102E30000E94C60A0E943B070E94F4070E940C08E9
:102E40000E9424080E943D089AC00E9424070E9404
:102E50003B070E9453070E946B070E9485070E9450
:102E6000BC070E94F4070E940C080E9424080E94DC
:102E70003D080E94550800913101002341F00230C5
:102E800031F0033021F0083011F00E946E0877C055
:102E90000E94A008F1E6ECED002319F00A95729665
:102EA000FBCF0E94D3080E94A508F6E6E2E000915D
:102EB0001E010A950A950A950A950A956FE1002365
:102EC00021F063950A957296FACFF0932401E0936E
:102ED00025010E94D308683211F40E94DE2408956F
:102EE0000E942D0D23C00E943C0D20C00E94B00DF9
:102EF0001DC00E94490D1AC00E94560D17C00E94A5
:102F0000630D14C00E94700D11C00E947D0D0EC093
:102F10000E943C040BC074FF05C0009135010E9463
:102F2000050D04C003C00E94960D00C00E949F22A0
:102F30006AE0089573FF04C00E949F226AE008952A
:102F400000911B010E94F10C1091260100911A01C1
:102F50000E94590C0E949F226AE008950E94A008D6
:102F6000F8E6E0EF0E94D3080E94A508F8E6E0EF3B
:102F70000E94D308009126010630F1F00EC00E9495
:102F8000A008F8E6E0EF0E94D3080E94A508F8E642
:102F9000E0EF0E94D30800912601002379F0013070
:102FA00019F1063038F0073031F0083021F00233E3
:102FB00021F0089559C06FC078C02CC060912601DF
:102FC0005F9A0E94900D0E94E70D0E94C30D0E941F
:102FD000CF0D0E94DB0D0E94A0090E94A008F3E61D
:102FE000EEE00E94D3080895609126015F9A0E9446
:102FF000900D0E94E70D0E94C30D0E94CF0D0E940C
:10300000DB0D0E94A008F9E6ECE00E94D3080E94C4
:103010009A0A0895609126015F9A0E94900D0E947D
:10302000E70D0E94C30D0E94CF0D0E94DB0D0E9490
:10303000A0090E94AE0E0E944B0D0E94A008F3E66C
:10304000EEE0FF96FF960E94D308F7E6E6EA0E94BC
:103050008503F7E6E8EB0E948503F7E6EAEC0E94B9
:1030600085030E94CE0E0895609126010E94C60A33
:103070000E94190D162F0E94450C009333010E94E7
:10308000BD0D0E94BA0A0E94DE0E0E94CE0E0027DD
:103090000093340108950E94A008F8E6E0EF0E9432
:1030A000D30867E00E949A0A0895609126010E9461
:1030B000E60E0E94F60E5F9A0E94900D0E94E70DA8
:1030C0000E94C30D0E94CF0D0E94DB0D0E94A0083C
:1030D000F3E6EEE0FC96F0960E94D3080E942C0BDB
:1030E0000E94A008F7E6EEE50E94D3080E94A5081A
:1030F000F7E6E0E70E94D3080E942C0B50E04CE07A
:1031000026E05093C5004093C4002093C200509322
:10311000CD004093CC002093CA00B1E1A6E30E9409
:10312000CE0E0E94610E0E94730E0E94ED0D0027CC
:103130000093090100930A0108956BE00E94762331
:10314000089575FF0C94D41900911E01002361F0BD
:10315000013029F0023021F0033019F0089549C000
:10316000F1C000C10E94000000911F01073009F466
:1031700002E3009326010E94BF0C063011F00E946A
:10318000970C0E949F226AE010911F01123080F17B
:10319000163071F1173061F11A951A950027F0E099
:1031A000E9E0E10FF01F0E94421200933101002775
:1031B000F0E0EDE0E10FF01F0E94421200933301B6
:1031C0000027F0E0E6E1E10FF01F0E9442120093B9
:1031D0001A010E94F60C00931B010027F0E0E2E1C7
:1031E000E10FF01F0E944212009332010E949D0ED7
:1031F0000895009120010E94C90C0430C0F400938E
:10320000330110912601112371F0123018F40E943D
:103210004F0C09C0163018F40E94390C04C0193044
:1032200010F40E944F0C0E949F226AE0089504301F
:1032300059F0053069F1063041F1073009F0089581
:103240006CE00E943A2408950E94A008FAE6EAE39E
:103250000E94D3080E94A508F8E6E0EF0E94D30878
:1032600000911C0110911D01011741F41395109359
:103270001D01143019F4112710931D010E940D0B2C
:1032800067E108950E94B50FCECF0E94200FCBCFEB
:103290000E94A008F9E6E2EF0E94D3080E94A50868
:1032A000F9E6EAEA0E94D3080E942C0B0E942C0B3C
:1032B0000E942C0B0E942C0B0E94A008F9E6ECEB5C
:1032C0000E94D3080E94A508F9E6EEEC0E94D308FC
:1032D0000E942C0B0E942C0B0E942C0B0E942C0B8A
:1032E0000E942C0B0E942C0B029913C0059911C04F
:1032F0000E94A008FAE6E8E20E94D3080E94A5080E
:10330000F9E6E0EE0E94D308F8940E942513789421
:103310008ACF0E94A008FAE6E4E00E94D3080E9447
:10332000A508FAE6E6E10E94D3080E942C0B0E9451
:103330002C0B0E942C0B0E942C0B0E942C0B0E9429
:103340002C0B71CF109126010091210100933101C6
:103350000E94230C009121010E94D30C0E949F2205
:103360006AE00895009122010E94DD0C10911F0176
:1033700000912201009332010E946F0C0E949D0E69
:103380000E949F226AE0089573FF04C06BE00E94D0
:1033900076230895F8940E94ED120E94B512789455
:1033A0006BE00E94762308956AE00E949F220091BC
:1033B00021010E94D30C0B2D11270E94850C0D2D8D
:1033C00011E00E94850C089575FF0C94F819009186
:1033D00023010023A9F00130D1F00230F9F00330CD
:1033E00021F1043049F1053071F1063099F1089569
:1033F0006BE00E947623009123010E94E70C089560
:103400000E94B50F10E008E350E140E029C00E949F
:10341000B50F10E008E354E040E222C00E94B50F6F
:1034200014E000E258E048E01BC00E94B50F18E02D
:1034300008E05BE040EF14C00E94B50F1BE000EF16
:1034400050E140E00DC00E94B50F10E000E050E0F8
:1034500048E306C00E94B50F10E000E050E140E0F4
:10346000312F202FB1E0A6E3A00FB11FF0E0E0E084
:10347000E00FF11F0C911C910E944A120117D1F725
:10348000112701E0200F311F31961196351791F762
:10349000241781F70E94160F0C947D050E944B1192
:1034A00065E10E9453120E94A009002700930401C5
:1034B000089576FF09C064E10E9453120E94A0099A
:1034C00000270093040108950E944B1100912601EA
:1034D000013029F0063020F0073019F0089584CD2E
:1034E000C3CDD9CD609326016AE00E949F22089542
:1034F000AA2475FD03C076FD07C0089560932601D8
:103500006AE00E949F220895613031F40E94900D7C
:1035100000922D0110922F016093260164E10E9418
:10352000A008F8E6EAEE0E94D308E0FC05C000908F
:103530002D0110902F0104C000902E011090300139
:103540000E9453120E94A00908950E94A0080093AF
:1035500026010E948A1080FDFCCF81FDFACF0E94D7
:10356000A508F8E6E6E30E94D3080E942C0B0E940F
:103570002C0B609326016AE00E949F2208950E940E
:103580002C0B0E942C0B0E94A008F8E6E0EF0E9492
:10359000D30867E00E949A0A70610E94910E089514
:1035A000AA2475FD03C077FD07C008956093260126
:1035B0006AE00E949F2208950E94900D00922D01C2
:1035C00010922F01609326017F7776FD06C068E098
:1035D0000E9453120E94A00908950E94A008F8E6D4
:1035E000E4EB0E94D30873FD07C00E94A508F8E62B
:1035F000E6EC0E94D30806C00E94A508F8E6E8EDB4
:103600000E94D308FFCFAA2475FD03C077FD07C031
:103610000895609326016AE00E949F2208950E9407
:10362000900D00922D0110922F01609326017F775B
:1036300067E00E9453120E94A0090895609326013A
:103640006AE00E949F22089582FD0C94431B83FD33
:103650000C94301B84FD0C945E1B85FD0C945A1B4E
:1036600037FC0C94391B339437FC33240E94AE0989
:103670000895032D0F77039507FD00270068302E6E
:103680000E94AE09089537FC0C944F1B032D0023B4
:1036900009F400E80A95302E0E94AE090895032D22
:1036A0000F77002309F400E80A950068302E0E9485
:1036B000AE09089543940E94C50908954A940E9452
:1036C000C5090895662319F0643151F00895082F53
:1036D000013021F0082F023011F0089509C03EC0DA
:1036E000082F013021F0082F0230C1F1089561C088
:1036F00010910401183031F0123009F00895716012
:103700000C94831B7260713039F07233A1F0753301
:10371000E9F07E7F7D7F08950E94A008F8E6E4E24C
:103720000E94D3080E94A508F8E6EAE50E94D308A3
:103730007061706208950E94A508F8E6E0EF0E94AB
:10374000D308746000270093040108950E94A5081F
:10375000F8E6EAE50E94D3087B7F08951091060100
:10376000183031F0123009F0089571600C94B91BD3
:103770007260713039F0723461F07534B1F07E7F6F
:103780007D7F0895132D1058312E0E94E00970643A
:1037900008950E94BE0800E20E94DB080E94DB0838
:1037A000746000270093060108950E94E0097B7F62
:1037B000089510910401183031F0123009F0089585
:1037C00071600C94E41B7260713039F0723551F005
:1037D0007535A1F07E7F7D7F08950E945312706140
:1037E000706408950BE80E94ED08F9E6E2E00E949B
:1037F000D308746000270093040108950E945312B7
:103800007B7F089582FD0C94231C83FD0C940F1C78
:1038100084FD0C944E1C85FD0C94421C089565316A
:1038200009F40895F0E0EDE1E00D08F4F395012DC1
:103830000E944A12002D0A3019F40027002E18C0E9
:103840000395002E15C0653109F40895F0E0EDE10F
:10385000E00D08F4F395012D0E944A12002D112766
:10386000011719F40AE0002E03C00A95002E00C0CB
:103870000E943511021511F008F00027102E0E9449
:10388000341D08950E943511012D122D011719F4D0
:103890000027102E0FC00395102E0CC00E9435116A
:1038A000012D1127011719F4022D102E03C00A95BE
:1038B000102E00C0613021F0653111F40E944B11CF
:1038C0000E94341D0895663028F0653151F068314A
:1038D00091F00895082F013059F0082F023059F067
:1038E0000895082F013029F0082F023019F00895AB
:1038F00003C063C08AC0D5C010910401183031F0F4
:10390000123009F0089571600C94871C7260713058
:1039100059F0723501F1753579F17233A9F17533CA
:10392000F1F17E7F7D7F0895D4FC12C0E1FC05C0DB
:10393000E0FC03C0D6FC0CC002C0D7FC09C00E944A
:10394000A508F8E6ECE60E94D3087061706408955B
:103950007062706124C00E94A508F8E6E0EF0E9442
:10396000D3087460002700930401A3940A2D033048
:1039700010F070627F7B08950E94A508F8E6ECE6DF
:103980000E94D3087B7F08950E94A508F8E6E0EF27
:103990000E94D308746000270093040108950E94D8
:1039A000A008F8E6E4E20E94D3080E94A508F8E621
:1039B000EAE50E94D3087B7F089510910401183036
:1039C00031F0123009F0089571600C94E81C7260B7
:1039D000713039F0723551F0753599F07E7F7D7F09
:1039E00008950E94A0097061706408950E94A5085E
:1039F000F8E6E0EF0E94D30874600027009304010A
:103A000008950E94A0097B7F089510910601183047
:103A100031F0123009F0089571600C94101D72603D
:103A2000713039F0723169F07531B1F07E7F7D7F90
:103A300008950E94A508F8E6EEE70E94D308706199
:103A400008950E94A508F8E6E0EF0E94D30874608C
:103A500000270093060108950E94A508F8E6EEE706
:103A60000E94D3087B7F0895002D0E94A10C012D98
:103A70000E94AB0C0E9453120E9416120E945E110B
:103A8000E00FF11F0E944212402E0E9416120E9467
:103A90007B11E00FF11F0E944212302E0E94A009FC
:103AA0000895613071F0D4FC0CC000913101002305
:103AB00041F0023031F0033021F0083011F0C0FC49
:103AC00001C050C010910601183031F0123009F0D9
:103AD000089571600C946D1D7260713039F0723808
:103AE00021F1753869F17E7F7D7F0895609326010D
:103AF00068E100913501009334010E94A008F9E6C5
:103B0000ECE20E94D308E0FC08C00E94A508F9E698
:103B1000E0E50E94D308706808950E94A508F9E6C0
:103B2000E2E60E94D308706808950E94A508F8E6AE
:103B3000E0EF0E94D3087460002700930601089507
:103B4000E0FC08C00E94A508F9E6E0E50E94D30861
:103B50007B7F08950E94A508F9E6E2E60E94D3085B
:103B60007B7F089510910601183031F0123009F072
:103B7000089571600C94BD1D7260713039F072331C
:103B8000A1F07533E9F07E7F7D7F08950E94A00843
:103B9000F8E6E4E20E94D3080E94A508F8E6EAE508
:103BA0000E94D3087061706208950E94A508F8E62B
:103BB000E0EF0E94D3087460002700930601089587
:103BC0000E94A508F8E6EAE50E94D3087B7F0895E5
:103BD00082FD0C94061E83FD0C94F51D84FD0C944F
:103BE000311E85FD0C94251E0895F0E0EDE1E00DF9
:103BF00008F4F395012D0E944A12002D0A3019F4A1
:103C00000027002E15C00395002E12C0F0E0EDE154
:103C1000E00D08F4F395012D0E944A12002D1127A2
:103C2000011719F40AE0002E03C00A95002E00C007
:103C30000E943511021511F008F00027102E0E9485
:103C4000F41EF4FE0E94910E08950E943511012D7C
:103C5000122D011719F40027102E0EC00395102EF7
:103C60000BC00E943511012D1127011719F4022DE7
:103C7000102E02C00A95102E0E94F41EF4FE0E941F
:103C8000910E0895673009F00895082F013021F052
:103C9000082F023011F0089501C053C010910401A3
:103CA000183031F0123009F0089571600C94591EEB
:103CB0007260713059F0723991F0753909F17233CF
:103CC00039F1753381F17E7F7D7F08950E94A508CB
:103CD000F8E6E0E90E94D3087061706808950E94D8
:103CE000A508F8E6E0EF0E94D3087460002700936F
:103CF0000401A3940A2D033010F070627F770895B9
:103D00000E94A508F8E6E0E90E94D3087B7F0895A9
:103D10000E94A508F8E6E0EF0E94D308746000272F
:103D20000093040108950E94A008F8E6E4E20E94CE
:103D3000D3080E94A508F8E6EAE50E94D3087B7F35
:103D4000089510910601183031F0123009F00895ED
:103D500071600C94AC1E7260713059F0723DC9F004
:103D6000753D39F17A3D69F17D3DB1F17E7F7D7F11
:103D700008950E94A008F8E6E4EB0E94D3080E9490
:103D8000A508F8E6E6EC0E94D308706170647068DC
:103D900008950E94A508F8E6E0EF0E94D308746039
:103DA000002700930601A3940A2D033008F07860E1
:103DB00008950E94A508F8E6E6EC0E94D3087B7FF0
:103DC00008950E94A508F8E6E0EF0E94D308746009
:103DD00000270093060108950E94A508F8E6E8ED83
:103DE0000E94D3087B7F0895002D0E94A10C012D15
:103DF0000E94AB0C0E9453120E9416120E945E1188
:103E0000E00FF11F0E944212402E0E9416120E94E3
:103E10007B11E00FF11F0E944212302E0E94A00978
:103E2000089582FD0C94311F83FD0C941E1F84FDA8
:103E30000C944C1F85FD0C94481F089537FC0C947E
:103E4000271F339437FC33240E94AE090895032DB5
:103E50000F77039507FD00270068302E0E94AE09FA
:103E6000089537FC0C943D1F032D002309F400E84E
:103E70000A95302E0E94AE090895032D0F77002376
:103E800009F400E80A950068302E0E94AE090895F2
:103E900043940E94C50908954A940E94C509089553
:103EA000683009F00895082F013021F0082F023002
:103EB00011F0089501C07BC010910401183031F059
:103EC000123009F0089571600C94671F72607130B0
:103ED00059F0723991F0753909F1723339F175334E
:103EE00081F17E7F7D7F08950E94A508F8E6E2EAD1
:103EF0000E94D3087061706808950E94A508F8E6D2
:103F0000E0EF0E94D3087460002700930401A3949B
:103F10000A2D033010F070627F7708950E94A50883
:103F2000F8E6E2EA0E94D3087B7F08950E94A50884
:103F3000F8E6E0EF0E94D3087460002700930401C4
:103F400008950E94A008F8E6E4E20E94D3080E94C7
:103F5000A508F8E6EAE50E94D3087B7F0895109152
:103F60000401183031F0123009F0089571600C949A
:103F7000BA1F7260713039F0723449F0753499F0BB
:103F80007E7F7D7F08950E945312706408950BE830
:103F90000E94ED08F9E6E2E00E94D3087460002771
:103FA0000093040108950E9453127B7F089510919D
:103FB0000601183031F0123009F0089571600C9448
:103FC000E21F7260713039F0723461F07534B1F013
:103FD0007E7F7D7F0895132D1058312E0E94E009B9
:103FE000706408950E94BE0800E20E94DB080E94EF
:103FF000DB08746000270093060108950E94E00921
:104000007B7F0895623309F00895082F013009F08D
:10401000089501C036C010910401183031F01230FB
:1040200009F0089571600C9416207260713039F0B7
:104030007233A1F07533E9F07E7F7D7F08950E9491
:10404000A008F8E6E4E20E94D3080E94A508F8E67A
:10405000EAE50E94D3087061706208950E94A50885
:10406000F8E6E0EF0E94D308746000270093040193
:1040700008950E94A508F8E6EAE50E94D3087B7F30
:10408000089510910601183031F0123009F00895AA
:1040900071600C944C207260713039F0723461F0B0
:1040A0007534B1F07E7F7D7F0895132D1058312E29
:1040B0000E94E009706408950E94BE0800E20E9418
:1040C000DB080E94DB087460002700930601089556
:1040D0000E94E0097B7F089582FD0C94802083FD7F
:1040E0000C94782084FD0C94902085FD0C948820FD
:1040F00000911A01039500931A010E94D50A0895B0
:1041000000911A010A9500931A010E94D50A089598
:1041100000911B01039500931B010E94F10A089571
:1041200000911B010A9500931B010E94F10A08955A
:10413000082F013021F0082F023051F1089510911D
:104140000401183031F0123009F0089571600C94B8
:10415000AA207260713039F0723139F0753181F016
:104160007E7F7D7F0895706108950E94A508F8E61E
:10417000E0EF0E94D30874600027009304010895C3
:104180000E94A5080E94D50A0E94F10A7B7F08952B
:1041900010910601183031F0123009F00895716065
:1041A0000C94D3207260713039F07A31A1F07D31F6
:1041B000E9F07E7F7D7F08950E94A008F8E6E4E2A2
:1041C0000E94D3080E94A508F8E6EAE50E94D308F9
:1041D0007061786008950E94A508F8E6E0EF0E94FB
:1041E000D308746000270093060108950E94A50873
:1041F000F8E6EAE50E94D3087B7F089582FD0C94DF
:10420000212183FD0C940A2184FD0C94472185FD16
:104210000C94382100911C010395043009F4002707
:1042200010911D01011741F4139510931D011430D5
:1042300019F4112710931D0100931C010E940D0B0E
:10424000089500911C010A95043008F003E01091D4
:104250001D01011741F4139510931D01143019F439
:10426000112710931D0100931C010E940D0B08954E
:1042700000911D010395043009F4002710911C01E1
:104280000117C1F300931D010E940D0B08950091C9
:104290001D010A95043008F003E010911C0101177C
:1042A000C1F300931D010E940D0B0895082F0130EA
:1042B00021F0082F023081F1089510910401183087
:1042C00031F0123009F0089571600C946821726029
:1042D000713039F0723169F07531B1F07E7F7D7FD8
:1042E00008950E94A508F7E6ECE40E94D3087061E7
:1042F00008950E94A508F8E6E0EF0E94D3087460D4
:1043000000270093040108950E94A508F7E6ECE455
:104310000E94D3087B7F089510910601183031F078
:10432000123009F0089571600C9497217260713019
:1043300039F07A31A1F07D31E9F07E7F7D7F0895FB
:104340000E94A008F8E6E4E20E94D3080E94A508B3
:10435000F8E6EAE50E94D3087061786008950E944B
:10436000A508F8E6E0EF0E94D308746000270093E8
:10437000060108950E94A508F8E6EAE50E94D30820
:104380007B7F089583FD0C94DD2185FD0C94DD2158
:1043900082FD0C94CF2184FD0C94CF2108950091CF
:1043A0001E010A95003110F000E10A95222712C083
:1043B00000931E010E949F22089500911E01039503
:1043C000003108F0002721E005C000931E010E9483
:1043D0009F220895109126011123A9F01130F1F0C8
:1043E00010913101112359F1113081F1123039F15D
:1043F000133029F1183079F135C0222391F2DFCF43
:104400002223B1F2E2CF0023D9F30830C9F30930F7
:10441000B9F30C30A9F30D3099F3EFCF002381F3FA
:10442000013071F3083061F3093051F30A3041F380
:104430000B3031F30C3021F30D3011F3DECF0430AB
:10444000E1F20530D1F20F30C1F2DACF0630A9F235
:10445000073099F2D5CF063081F2073071F20F3074
:1044600061F2CECF043049F2053039F2063029F23C
:10447000073019F2C5CF082F023029F0082F01307C
:1044800009F0089536C010910601183031F012304D
:1044900009F0089571600C944E227260713039F009
:1044A0007231A1F07531E9F07E7F7D7F08950E9421
:1044B000A008F8E6EAE50E94D3080E94A508F8E6FD
:1044C000E6E30E94D30870617F7D08950E94A508ED
:1044D000F8E6E0EF0E94D30874600027009306011D
:1044E00008950E94A508F8E6E6E30E94D3087B7FC2
:1044F000089510910401183031F0123009F0089538
:1045000071600C9484227260713039F0723349F01A
:10451000753391F07E7F7D7F089511D07061706258
:1045200008950E94A508F8E6E0EF0E94D3087460A1
:1045300000270093040108951DD07B7F08950E94F9
:10454000A008F9E6E4E70E94D30808E80E94ED0815
:1045500000911E01093020F400E30E94DB080AC02C
:1045600001E30E94DB0800911E0117E2010F0E9487
:10457000DB0806C000911E0111E3010F0E94DB0859
:104580000E94A508F0E6EAEA00911E01002319F056
:104590000A957296FBCF0E94D30808950808090572
:1045A000F5E4ECE900911E011127E00FF11F549191
:1045B000F1E0EFE1E00FF11F408183FD0C94F02268
:1045C00085FD0C94F02282FD0C94EA2284FD0C946B
:1045D000EA2208954A95451738F0452F4A9504C0B8
:1045E0004395451708F04427F1E0EFE100911E01E3
:1045F0001127E00FF11F40830E9489230895082F9F
:10460000023031F0082F013009F0089540C00895BC
:1046100010910601072F183031F0123009F008957B
:1046200001600C9415230260702F013041F00231BB
:10463000B9F0053111F10E7F0D7F702F08950E94A2
:10464000A008F8E6E4E20E94D3080E94A508F8E674
:10465000EAE50E94D308072F00610F7D702F0895AF
:104660000E94A508F8E6E0EF0E94D308072F046037
:10467000702F00270093060108950E94A508F8E610
:10468000EAE50E94D308072F0B7F702F0895109141
:104690000401072F183031F0123009F0089501603D
:1046A0000C9454230260702F013041F0023361F00A
:1046B0000533B9F00E7F0D7F702F089517D0072FA7
:1046C00000610062702F08950E94A508F8E6E0EFEF
:1046D0000E94D308072F0460702F00270093040165
:1046E000089517D0072F0B7F702F08950E947B230A
:1046F0000E94892308950E94A008F1E6ECED009144
:104700001E01002319F00A957296FBCF0E94D30870
:10471000089500911E01003039F0013061F002303F
:1047200089F00330B1F008950E94A508F3E6EEE0A9
:1047300000911F0115C00E94A508F3E6E0EB00916F
:1047400020010EC00E94A508F4E6E2E500912101D7
:1047500007C00E94A508F5E6E6E00091220100C02E
:10476000002319F00A957296FBCF0E94D308089592
:1047700083FD0C94D12385FD0C94D12382FD0C94F0
:10478000C52384FD0C94C5230895009123010A9547
:10479000073010F007E00A95009323010E943A24A5
:1047A0000895009123010395073008F00027009336
:1047B00023010E943A240895082F023029F0082F7F
:1047C000013009F0089530C010910601183031F021
:1047D000123009F0089571600C94EF23726071300B
:1047E00039F0723171F07531B9F07E7F7D7F0895B7
:1047F0000E94A508F8E6E6E30E94D30870617F7D79
:1048000008950E94A508F8E6E0EF0E94D3087460BE
:1048100000270093060108950E94A508F8E6E6E344
:104820000E94D3087B7F089510910401183031F065
:10483000123009F0089571600C941F247260713079
:1048400039F0723349F0753391F07E7F7D7F0895A2
:1048500011D07061706208950E94A508F8E6E0EF3B
:104860000E94D3087460002700930401089502D0C9
:104870007B7F08950E943F240E944D2408950E944A
:10488000A008F3E6E0EB00912001002319F00A955F
:104890007296FBCF0E94D30808950E94A508F5E602
:1048A000E2E700912301002319F00A957296FBCFED
:1048B0000E94D3080895082F013021F0082F0230FC
:1048C00041F0089510910401183069F0123041F060
:1048D000089510910601183059F1123031F1089500
:1048E00071600C9474247260713039F0723141F04F
:1048F000753189F07E7F7D7F089570617F7708959F
:104900000E94A508F9E6E2E00E94D308746000273F
:104910000093040108950E94A508F0912401E091FC
:1049200025010E94D3087B7F089571600C9499241F
:104930007260713039F0723851F0753899F07E7FBD
:104940007D7F08950B2DB02E70687F7E08950E94A4
:10495000BE08F9E6E2E00E94D308746000270093E5
:10496000060108950E94A508F0912401E091250117
:104970000E94D3087B7F089582FD0C94D32483FD8D
:104980000C94C82484FD0C94D32485FD0C94C82475
:104990000091350103950B3009F401E000933501D6
:1049A0000E94DE240895009135010A95002309F440
:1049B0000AE0009335010E94DE2408950CEC0E9469
:1049C000ED08009135010A3038F001E30E94DB0860
:1049D00000E30E94DB08089500E30E94DB080091D9
:1049E000350110E3010F0E94DB080895082F013004
:1049F00021F0082F023061F1089510910401183060
:104A000031F0123009F0089571600C94082572603D
:104A1000713039F0723139F0753181F07E7F7D7FF0
:104A20000895706108950E94A508F8E6E0EF0E94DD
:104A3000D308746000270093040108950E94A5081C
:104A4000F7E6EAE30E94D3080E94DE247B7F089504
:104A500010910601183031F0123009F0089571609C
:104A60000C9433257260713039F07A31A1F07D31C8
:104A7000E9F07E7F7D7F08950E94A008F8E6E4E2D9
:104A80000E94D3080E94A508F8E6EAE50E94D30830
:104A90007061786008950E94A508F8E6E0EF0E9432
:104AA000D308746000270093060108950E94A508AA
:104AB000F8E6EAE50E94D3087B7F0895D2FE01C0A4
:104AC0005AC00091170110911901011709F029C06E
:104AD000663021F1673011F1683001F16233F9F08D
:104AE00020913101222309F46BC1223009F468C1FD
:104AF000213009F497C2233009F48BC3243009F420
:104B00008EC4253009F417C5263009F488C427302F
:104B100009F4C9C5283009F477C60895E5C70C948F
:104B2000662E663021F1673011F1683001F1623391
:104B300001F120913101002309F4C8C1223009F4A8
:104B4000C5C1213009F4D9C2233009F4B1C32430DE
:104B500009F47EC4253009F42AC5263009F478C446
:104B6000273009F4E0C5283009F4DFC608950C9415
:104B7000A02D0C94CD2E0091160110911801011753
:104B800009F01EC020913101222309F4ACC122306A
:104B900009F4A9C1213009F4BDC2233009F495C339
:104BA000243009F460C4253009F40CC5263009F41A
:104BB0005AC4273009F4C2C5283009F4C3C6089581
:104BC00020913101222309F420C2223009F41DC2B0
:104BD000213009F410C3233009F414C4243009F43B
:104BE0009FC4253009F454C5263009F499C42730F0
:104BF00009F4FFC5283009F469C708950E94C30D60
:104C0000552400270093340100913101002339F02D
:104C1000023029F0033019F0083009F001C05EC0FD
:104C20000E9467154F935F930E9498115F914F9177
:104C30005093290140932A0100922D0110922F01D7
:104C40000FEF0015010519F40E94C90D03C00E9461
:104C5000CF0D00C00E942D260895D4FCACC0E0FC0E
:104C600003C0D6FCA6C002C0D7FCA3C05093290144
:104C700040932A0100922D0110922F0108C05093F9
:104C80002B0140932C0100922E0110923001E0FC88
:104C900009C000902D0110902F010E94410E0E942A
:104CA000990A08953091290120912A0150912B01F0
:104CB00040912C01421B530B11F022F432F00E9460
:104CC000490E05C00E94510E02C00E94590E00906C
:104CD0002E01109030010E94990A0895E5FC03C04E
:104CE000E6FC1BC008950E9467154F935F930E94D6
:104CF00098115F914F915093290140932A0100929E
:104D00002D0110922F010FEF0015010519F40E94DB
:104D1000C90D1DC00E94CF0D1AC00E9467154F9388
:104D20005F930E9498115F914F9150932B01409394
:104D30002C0100922E01109230010FEF0015010599
:104D400019F40E94D50D03C00E94DB0D00C00E9423
:104D5000AA260895D4FC2FC0E1FC0DC0D6FC29C0C2
:104D6000E6FC089500902D0110902F010E94410E45
:104D70000E94990A0895D7FC1CC030912901209106
:104D80002A0150912B0140912C01421B530B11F031
:104D900022F432F00E94490E05C00E94510E02C05A
:104DA0000E94590E00902E01109030010E94990A25
:104DB00008950E94C60A0E94410E0E94BA0A0895F0
:104DC000F1E1E6E33FEF1127222733950091170128
:104DD000301730F00E94EF14C1FC0E94F3130895C5
:104DE0000191033209F40081013408F4EECF0B3550
:104DF00008F0EBCF132F339500911701301718F0FF
:104E00000E94EF14089501910B33A9F7232F121775
:104E100008F00895022F011B063208F00895FF9351
:104E2000EF93F1E1E6E30027E10FF01FFF93EF932B
:104E3000D1FE0DC00191063451F40191013439F4D1
:104E400000810B3321F406E4029309E40293EF910D
:104E5000FF9101910B33E9F7022F011B0D3019F07F
:104E6000033009F051F5F1E1E6E30027E10FF01F0F
:104E70000191063411F50081043579F0013419F0FF
:104E8000023431F01AC00E941D0E0E942F0E18C06D
:104E90000E94230E0E94290E13C031960081013317
:104EA00031F00E943B0E0E94900D319706C00E9487
:104EB000350E0E948A0D319700C0EF91FF9185CF8A
:104EC00034963F930E94FE253F91F7CFF1E1E6E350
:104ED000002710911901E10FF01F112722273091AF
:104EE00019013A9572CFF2E1E6E33FEF112722274D
:104EF000339500911601301708F00895019103329F
:104F000009F40081013408F4F3CF0B3508F0F0CF39
:104F1000132F339500911601301718F00E94EF14EB
:104F2000089501910B33A9F7232F121708F0089564
:104F3000022F011B063208F00895FF93EF93F2E170
:104F4000E6E30027E10FF01F01910B33E9F7022F91
:104F5000011B053229F00D3019F0033009F047C06C
:104F6000F2E1E6E30027E10FF01F0191093421F09F
:104F70000634D9F03CC03BC000810634E1F70E9402
:104F80001D0E0E942F0EFF93EF937F960081EF91ED
:104F9000FF91013329F40E94350E0E948A0D2AC028
:104FA0000E943B0E0E94900D25C00081043579F0CF
:104FB000013419F0023431F01AC00E941D0E0E9413
:104FC0002F0E18C00E94230E0E94290E13C0319686
:104FD0000081013331F00E943B0E0E94900D319709
:104FE00006C00E94350E0E948A0D319700C0EF91D5
:104FF000FF917ECF349600911701002309F0F7CF7F
:105000003F930E94FE253F91F2CFF2E1E6E30027B5
:1050100010911801E10FF01F11272227309118017C
:105020003A9566CFF1E1E6E33FEF1127222733956A
:1050300000911701301718F00E94EF1408950191A4
:105040000E3F21F4132F01913395F1CF0D3F79F7E6
:10505000232F121708F00895022F011B0B3008F0C0
:105060000895FF93EF93F1E1E6E30027E10FF01FCE
:1050700001910D3FE9F7022F011B0A3091F4F1E194
:10508000E6E30027E10FF01F01910E3F01910E3F73
:1050900032960191003041F0033031F0053021F0BB
:1050A00000C0EF91FF91C3CF339600810F9302951B
:1050B0000F7010E3010F009311010F910F70010F9A
:1050C00000931201319700810F9302950F70010F29
:1050D000009313010F910F70010F0093140131978A
:1050E000008102950F70010F00931501F1E0E1E1DD
:1050F0003F930E94FE253F91D4CFF1E1E6E30027E4
:1051000010911901E10FF01F112722273091190189
:105110003A958DCFF2E1E6E33FEF11272227339551
:1051200000911601301708F0089501910E3F21F407
:10513000132F01913395F3CF0D3F89F7232F1217CA
:1051400008F00895022F011B0B3008F00895FF931B
:10515000EF93F2E1E6E30027E10FF01F01910D3F2D
:10516000E9F7022F011B063009F414C00A3091F44C
:10517000F2E1E6E30027E10FF01F01910E3F0191FC
:105180000E3F32960191003041F0033031F005308E
:1051900021F000C0EF91FF91C2CF339600810F93B1
:1051A00002950F7010E3010F009311010F910F7022
:1051B000010F00931201319700810F9302950F7038
:1051C000010F009313010F910F70010F0093140151
:1051D0003197008102950F70010F00931501F1E0E6
:1051E000E1E100911701002309F0D4CF3F930E9421
:1051F000FE253F91CFCFF2E1E6E3002710911801A1
:10520000E10FF01F11272227309118013A9587CF1F
:105210000895F1E1E6E33FEF11272227339500914E
:105220001701301730F00E94EF14C1FC0E94F313F5
:1052300008950191013408F4F1CF0B3508F0EECF59
:10524000132F339500911701301718F00E94EF14B7
:10525000089501910B33A9F7232F121708F0089531
:10526000022F011B0C3108F00895FF93EF93F1E139
:10527000E6E30027E10FF01FFF93EF93D1FE0DC08F
:105280000191063451F40191013439F400810B335A
:1052900021F406E4029309E40293EF91FF91019156
:1052A0000B33E9F7022F011B01F4EF91FF91B6CF09
:1052B000F1E1E6E3002710911901E10FF01F11273A
:1052C0002227309119013A95A9CFF2E1E6E33FEFA9
:1052D00011272227339500911601301708F0089501
:1052E0000191013408F4F6CF0B3508F0F3CF132FFA
:1052F000339500911601301718F00E94EF140895AD
:1053000001910B33A9F7232F121708F00895022FEC
:10531000011B0C3108F00895FF93EF93F2E1E6E3EF
:105320000027E10FF01F01910B33E9F7022F011B5A
:10533000502F0A3149F00B3139F00A3029F00B3087
:1053400019F0033009F04BC0F2E1E6E30027E10F6A
:10535000F01F0191093469F00634E9F00F3409F0C7
:105360003EC000810934E1F70E94230E0E94290EFD
:1053700007C000810634A1F70E941D0E0E942F0E67
:10538000FF93EF9378965B3109F431960081EF91AA
:10539000FF91339627C00081043589F0013419F05C
:1053A000023439F01CC00E941D0E0E942F0E30974F
:1053B00019C00E94230E0E94290E309713C0319607
:1053C0000081013331F00E943B0E0E94900D319715
:1053D00006C00E94350E0E948A0D319700C0EF91E1
:1053E000FF9178CF31965A3119F05A3009F0319641
:1053F00000911701002309F0F2CF3F930E94FE2590
:105400003F91EDCFF2E1E6E3002710911801E10FA3
:10541000F01F11272227309118013A955BCFF1E157
:10542000E6E33FEF00911701053029F00A3009F05B
:10543000089559E001C054E03395009117013017E9
:1054400018F00E94EF14089501913517A1F7F3CFDA
:10545000F1E1E6E3002710911901E10FF01F30910F
:1054600019013A95E8CFF2E1E6E33FEF009116012A
:10547000053029F0073009F0089556E001C054E0E6
:10548000339500911601301718F00E94EF1408951B
:1054900001913517A9F7563011F433970191003077
:1054A000C9F00130B9F00230A9F0033099F00430AE
:1054B00089F0063079F0083069F0023859F0033885
:1054C00049F0043839F0083829F00A3019F00C3066
:1054D00009F0D5CF359701910F7010E3010F0093BC
:1054E000110101910F9302950F70010F00931201AA
:1054F0000F910F70010F0093130100810F9302951C
:105500000F70010F009314010F910F70010F0093A2
:105510001501F1E0E1E13F930E94FE253F91AFCFFD
:10552000F2E1E6E3002710911801E10FF01F30913E
:1055300018013A95A4CFF1E1E6E33FEF009117019E
:10554000053011F008953596339500911701301705
:1055500018F00E94EF14089501913430A9F70A3031
:1055600099F7329700810F7010E3010F009311013A
:1055700002910F9302950F70010F009312010F918A
:105580000F70010F0093130102910F9302950F709A
:10559000010F009314010F910F70010F009315017B
:1055A000F1E0E1E13F930E94FE253F91CDCFF1E193
:1055B000E6E3002710911901E10FF01F3091190166
:1055C0003A95C2CFF2E1E6E33FEF009116010031D8
:1055D00019F0003209F00895339500911601301743
:1055E00018F00E94EF14089501913430A9F7F2E108
:1055F000E6E30081013308F0EFCF3F932F921F9233
:105600000F92F2E1E6E3319601910F700295102FAF
:1056100001910F93007F0295010F202E0F910F70C3
:105620000295102F01910F93007F0295010F102E0C
:105630000F910F700295102F0191007F0295010FBD
:10564000002E0E9440150F901F902F9040E3032FD3
:105650000F70040F00931101022F007F0295040FB9
:1056600000931201022F0F70040F00931301012FFA
:10567000007F0295040F00931401012F0F70040F97
:1056800000931501F1E0E1E10E94FE253F91A4CFD6
:10569000F2E1E6E3002710911801E10FF01F3091CD
:1056A00018013A9599CFF1E1E6E33FEF0091170138
:1056B000053021F00A3009F00895359633950091B0
:1056C0001701301718F00E94EF140895019134303B
:1056D000A9F70A3099F7349701910F930F7010E3EF
:1056E000010F009315010F9102950F70010F0093A8
:1056F000140101910F930F7010E3010F0093130138
:105700000F9102950F70010F0093120100810F702D
:1057100010E3010F00931101F1E0E1E13F930E94DA
:10572000FE253F91CBCFF1E1E6E30027109119016F
:10573000E10FF01F309119013A95C0CFF2E1E6E395
:105740003FEF009116010E3029F00C3119F00432B0
:1057500009F00895339500911601301718F00E9452
:10576000EF14089501913430A9F7F2E1E6E30081E6
:10577000013308F0EFCF3F93F2E1E6E33196419138
:10578000319121911191FF93EF93DF93CF93CAE071
:10579000DD270E947C16CF91DF91EF91FF91012EC2
:1057A000122E232E0E94401540E3032F0F70040F8A
:1057B00000931101022F007F0295040F0093120144
:1057C000022F0F70040F00931301012F007F029529
:1057D000040F00931401012F0F70040F00931501A3
:1057E000F1E0E1E10E94FE253F91F2E1E6E335962A
:1057F000B1CFF2E1E6E3002710911801E10FF01FAD
:10580000309118013A95A6CFF1E1E6E33FEF112779
:105810002227339500911701301718F00E94EF14DA
:10582000089501910E3F21F4132F01913395F1CF8B
:105830000D3F79F7232F121708F00895022F011B4F
:105840000B3008F00895FF93EF93F1E1E6E30027B2
:10585000E10FF01F01910D3FE9F7022F011B0A3004
:1058600019F00B3099F059F5F1E1E6E30027E10F6B
:10587000F01F01910E3F01910E3F329601910030D1
:1058800009F10330F9F00530E9F019C0F1E1E6E380
:105890000027E10FF01F01910E3F01910E3F32965C
:1058A00001910C3121F40191033089F008C00532D7
:1058B00031F40191003031F0013049F000C0EF9136
:1058C000FF91A7CF0E941D0E0E942F0ED1C00E94F3
:1058D000230E0E94290ECCC0339600810F930295AF
:1058E0000F7010E3010F009311010F910F70010F62
:1058F00000931201319700810F9302950F70010FF1
:10590000009313010F910F70010F00931401319751
:10591000008102950F70010F00931501F1E0E1E1A4
:105920003F930E94FE253F91CACFF1E1E6E30027B5
:1059300010911901E10FF01F112722273091190151
:105940003A9567CFF2E1E6E33FEF1127222733953F
:1059500000911601301708F0089501910E3F21F4CF
:10596000132F01913395F3CF0D3F89F7232F121792
:1059700008F00895022F011B0C3008F00895FF93E2
:10598000EF93F2E1E6E30027E10FF01F01910D3FF5
:10599000E9F7022F011B073039F00630D9F10A3040
:1059A00021F00B30A1F061C060C0F2E1E6E3002716
:1059B000E10FF01F01910E3F01910E3F32960191D0
:1059C0000030F1F00330E1F00530D1F04EC0F2E1EB
:1059D000E6E30027E10FF01F01910E3F01910E3F1A
:1059E000329601910C3121F40191033071F0E9F507
:1059F0000532D9F50191003019F0013031F035C090
:105A00000E941D0E0E942F0E33C00E94230E0E9482
:105A1000290E2EC0F2E1E6E30027E10FF01F01910D
:105A20000E3F01910E3F329601910F3009F01DC0DB
:105A30000081002369F40E94230E0E942F0E0E9411
:105A40003B0E0E94900D009117010023D1F10DC073
:105A50000E94230E0E942F0E0E94350E0E948A0D76
:105A600000911701002369F100C0EF91FF916FCF02
:105A7000339600810F9302950F7010E3010F00938E
:105A800011010F910F70010F0093120131970081E6
:105A90000F9302950F70010F009313010F910F7078
:105AA000010F009314013197008102950F70010FCF
:105AB00000931501F1E0E1E100911701002309F0E5
:105AC000D4CF3F930E94FE253F91CFCFF2E1E6E392
:105AD000002710911801E10FF01F112722273091A4
:105AE00018013A9534CF0895F1E1E6E33FEF33959D
:105AF00000911701301708F00895F0FE0FC00091D3
:105B00001701093051F40E949916002331F40E94C4
:105B1000670E0E946D0E0E94F914089500911701FE
:105B2000053169F4F1E1E6E3109117010E94AD2D12
:105B3000F2FE08950E947F0E0E94C02D08950895E0
:105B4000F1E1E6E3002710911901E10FF01F1127A1
:105B50002227309119013A95CACFF1E1E6E301918C
:105B6000063069F40191023151F401910D3E39F48E
:105B70000E948F16002319F40E94790E089508954B
:105B8000F1E1E6E33A960191003810F40BE201C02E
:105B90000DE200934F132F933F934F935F93219107
:105BA0003191419151918894221F331F441F551FF9
:105BB0008894563828F4553820F0403910F000C049
:105BC0007EC05F57552311F401E007C001E08894BF
:105BD000001F5150552309F0FBCF009350130027AD
:105BE000009355130093541300E1009353134F9304
:105BF00042954F7000915313402B409353134F9194
:105C00004295407F409352133F9332953F700091ED
:105C10005213302B309352133F913295307F309393
:105C2000511304E60E94CA15009150130E94CA1530
:105C300040915513309154132091531310915213E6
:105C40000091511388944795379527951795079597
:105C50008894479537952795179507958894479584
:105C600037952795179507958894479537952795E4
:105C700017950795132F022F0E94FD1510E3032F90
:105C800002950F70010F00933F13032F0F70010F48
:105C900000933E13022F02950F70010F00933D13E6
:105CA000022F0F70010F00933C135F914F913F91B2
:105CB0002F910E94790EF4FC0E94970E08950E9485
:105CC000850E5F914F913F912F910895F1E1E6E3A9
:105CD0003FEF11272227339500911701301710F05D
:105CE0000C94DA2E01910A3209F0F5CF132F339577
:105CF00000911701301710F00C94DF2E01910A303B
:105D0000B1F7232F121710F00C94E42EF1E1E6E323
:105D10000027E10FF01F01910A30E9F7022F011B64
:105D2000502F5A95F1E1E6E300275F93F1E1E6E3B6
:105D3000002700810A3219F05F910C94E82E01913E
:105D40005A955523E1F7033219F05F910C94ED2E2B
:105D50000E941D2F002319F45F910C94F22E5F9185
:105D60005A955A95F1E1E6E300270191008100354B
:105D700069F0013461F0043559F0083451F003350D
:105D800049F00B3441F0023539F008957BC0B5C0BD
:105D90008DC09CC0E1C0AAC073C1F1E1E6E3002759
:105DA00010911901E10FF01F1127222730911901DD
:105DB0003A9591CFFAE6EEEC0E9485030895FAE653
:105DC000EAEE0E9485030895FBE6E2E30E94850364
:105DD000FBE6E2E60E9485030895FBE6E0E70E9409
:105DE00085030895FBE6EEE70E94850300C0F1E11C
:105DF000E6E3002701910E947C035A955523D1F7D1
:105E00000DE00E947C030AE00E947C030895FBE6FB
:105E1000EAE90E948503F1E1E6E3002753955395F3
:105E200001910E947C035A955523D1F70DE00E9401
:105E30007C030AE00E947C030895FBE6E6EA002763
:105E40004FEF439505910532E1F7FBE6E6EA33278C
:105E5000B1E1A6E357E03395341791F00D91159118
:105E6000011729F45A955523B1F701E00895FBE68F
:105E7000E6EA0027E30FF01FB1E1A6E357E0EBCF1E
:105E800000270895F1E1E6E30027E50FF01F008108
:105E9000003319F45F9ABBDF0895013319F45F985A
:105EA000B6DF0895539553950C94F22EF1E1E6E395
:105EB000002735960081003511F00C94F22E032D49
:105EC0000F77302E0E94E009A2DF0895F1E1E6E3AA
:105ED000002735960081003511F00C94F22E032D29
:105EE0000068302E0E94E00992DF0895052F5A3095
:105EF00011F05B3009F06DC0AEC0F1E1E6E31127AF
:105F00000027379601910053033030F00C94A82FEE
:105F1000539553950C94F22E002331F0013019F46F
:105F200014E60C94942F18EC019100530A3010F0F1
:105F30000C94F22E2AE0029F100D019100530A30BA
:105F400010F00C94F22E100F10930D0160DF0895E5
:105F5000539553950C94F22EF1E1E6E311270027B7
:105F6000389601910053023030F00C94E52F539590
:105F700053950C94F22E002331F0013019F414E6FD
:105F80000C94C32F18EC019100530A3020F0539564
:105F900053950C94F22E2AE0029F100D01910053AC
:105FA0000A3020F0539553950C94F22E8894100FDC
:105FB000103820F0539553950C94F22E312E5F93A8
:105FC0000E94AE095F9123DF0895539553950C9479
:105FD000F22EF1E1E6E311270027389601910053F4
:105FE000033030F00C942730539553950C94F22ED7
:105FF000002331F0013019F414E60C94003018EC51
:10600000019100530A3020F0539553950C94F22ED1
:106010002AE0029F8894100D20F4539553950C9418
:10602000F22E019100530A3020F0539553950C94B1
:10603000F22E8894100F20F4539553950C94F22E61
:10604000412E5F930E94C5095F91E1DE089553954B
:1060500053950C94F22EF1E1E6E300273996008186
:10606000013431F00E3441F0539553950C94F22ED7
:106070000E944F0DCCDE08950E944B0DC8DE08959E
:10608000F1E1E6E3002736960081033211F00C942B
:10609000F22EBDDE0E940000FFFFFFFFFFFFFFFFAB
:1060A000FFFFFFFFFFFFFFFF00002020426574722B
:1060B0006965622F4D6F646520200000202020203C
:1060C00053706569636865722020202000002020DD
:1060D0005472616E736365697665722020200000DA
:1060E0002020202042617564726174652020202088
:1060F00000002020202049434F4D2D4944202020DE
:106100002020000020202020202043492D56202040
:106110002020202000002020204641202D2D2D3E33
:106120002049462020200000202020464220736580
:106130006E64656E202020200000202020205665FF
:106140007273696F6E202020202000002020202004
:10615000432D5765727465202020202000002020E8
:10616000202042616E64706C616E2020202000004F
:106170002020205054542D52656C616973202020DA
:10618000000020202020496E666F746578742020FE
:1061900020200000496E666F746578742D41757318
:1061A000676162650000202020506F6C6C2D50618B
:1061B000757365202020000020202053706C6974C6
:1061C0002F4D656EF520202000002A2A204572728E
:1061D0006F72205B30305D202A2A00002D2042653E
:1061E00074726965622F4D6F6465202D00002D204B
:1061F000202053706569636865722020202D00009F
:106200002D205472616E7363656976657220202D4E
:1062100000002D2020204261756472617465202089
:10622000202D00002D20202049434F4D2D49442092
:106230002020202D00002D202020202043492D56F5
:1062400020202020202D00002D20204641202D2D13
:106250002D3E20494620202D00002D2020464220A2
:1062600073656E64656E2020202D00002D20202097
:1062700056657273696F6E202020202D00002D203E
:106280002020432D5765727465202020202D0000AA
:106290002D20202042616E64706C616E2020202DC4
:1062A00000002D20205054542D52656C61697320DC
:1062B000202D00002D202020496E666F74657874B3
:1062C0002020202D00002020202020202020202001
:1062D00020202020202000002D2020506F6C6C2DCD
:1062E000506175736520202D00002D202053706CA7
:1062F00069742F4D656EF520202D00002A2A204557
:1063000072726F72205B30315D202A2A00002020DB
:1063100020204D616E75656C6C20202020200000CF
:10632000202020205370656963686572202020203A
:106330000000205472616E73636569766572202077
:1063400031200000205472616E7363656976657256
:10635000202032200000205472616E7363656976DC
:106360006572202033200000205472616E736365D3
:106370006976657220203420000020202041412DC4
:106380005A65726F204949202020000020202020DB
:106390002052656D6F7465202020202000002A2A7D
:1063A000204572726F72205B30325D202A2A000015
:1063B00020537065696368657262616E6B2031207D
:1063C000000020537065696368657262616E6B20BE
:1063D0003220000020537065696368657262616EE7
:1063E0006B2033200000205370656963686572621A
:1063F000616E6B20342000005370656963682E2045
:106400006B6F70696572656E0000537065696368D3
:106410006572206CEF736368656E000020446174E0
:10642000656E736963686572756E6720000020444D
:106430006174656E2065696E6C6573656E20000021
:106440002A2A204572726F72205B30335D202A2A1F
:10645000000020202020456C656372616674202056
:106460002020000020202049434F4D2028616C74DB
:10647000292020200000202020204B656E776F6FA0
:1064800064202020202000002020202046542D328F
:1064900030303020202020200000202020204654B2
:1064A0002D383137202020202020000020202046B9
:1064B000542D313030304D5020202020000020203D
:1064C000202046542D383437202020202020000062
:1064D0002020202046542D3932302020202020201A
:1064E000000020202049434F4D20286E657529204B
:1064F000202000002A2A204572726F72205B3035FE
:106500005D202A2A00002034383030206264202D9B
:106510002038204E2031000020393630302062648F
:10652000202D2038204E20310000313932303020EB
:106530006264202D2038204E203100003338343062
:1065400030206264202D2038204E2031000020347D
:10655000383030206264202D2038204E2032000058
:106560002A2A204572726F72205B30365D202A2AFB
:106570000000537065696368657262616E6B2031FB
:106580002D34000020537065696368657262616E26
:106590006B2031200000205370656963686572626A
:1065A000616E6B203220000020537065696368655E
:1065B0007262616E6B203320000020537065696346
:1065C00068657262616E6B20342000002045696E40
:1065D0007374656C6C756E67656E202000002020FA
:1065E000766F6C6C7374E16E646967202020000024
:1065F0002A2A204572726F72205B30345D202A2A6D
:106600000000696E7465726E2020202065787465C4
:10661000726E00006A61202020202020202020208F
:106620006E65696E00006A612020202020202020F5
:1066300020206E65696E00006E6575202020202088
:106640002020202020616C74000037393620202063
:10665000202020202020323535300000444C2020DE
:1066600020202020202020202020444B00006A6190
:10667000202020202020202020206E65696E000030
:106680006A61202020202020202020206E65696E55
:1066900000006A61202020202020202020206E651C
:1066A000696E0000202053656B756E64656E3A203C
:1066B00020202020000053706C69742020202020AE
:1066C00020204D656EF500002A2A204572726F72F7
:1066D000205B30375D202A2A0000696E7465726E77
:1066E000000065787465726E000020206A612020C9
:1066F0000000206E65696E200000206E6575202008
:10670000000020616C7420200000203739362020E2
:10671000000020323535302000002020444C20205D
:1067200000002020444B2020000053706C6974202E
:106730000000204D656EF5200000202053656B752C
:106740006E64656E3A20202020200000206B6F7060
:10675000696572656E206CE175667420000020200A
:106760002041412D5A65726F2049492020200000A8
:106770002076657262696E64656E202E2E2E2E2044
:1067800000003C50524553533E20202020203C4FD7
:106790004B3E000020444C334C41432D4B6F7070F6
:1067A0006C6572200000436F6E74726F6C6C657262
:1067B0002056362E30300000202843292031382E34
:1067C00030352E32303236200000646C3968646116
:1067D00040646C396864612E646500002D2D20547E
:1067E00057492D4552524F5231202D2D00002D2D4D
:1067F000205457492D4552524F5232202D2D000022
:106800002D2D205457492D4552524F5233202D2DB6
:1068100000002D2D205457492D4552524F523420FF
:106820002D2D0000205765636873656C20696E200C
:106830006461732000007769656465722076657213
:106840006C617373656E000020446174656E206531
:10685000696E6C6573656E2000002020202D2D2050
:106860004D656EF5202D2D20202000002020202DAC
:106870002D2045444954202D2D202020000020208B
:10688000202D2D20454E4445202D2D202020000078
:1068900020202D2D2052656C616973202D2D202024
:1068A0000000202D2D204672657175656E7A202DB1
:1068B0002D200000416E70617373756E67206669EC
:1068C0006E64656E0000202D2D2046726571756521
:1068D0006E7A202D2D2000002020202D2D204261B9
:1068E0006E64202D2D2020200000454449542000B6
:1068F0002020202020202020202020202020202098
:106900000000202020202020202000004D454D2088
:1069100020202020202020005452580044525800AB
:106920002020202000002A2A2A2A2A002020537012
:106930006C69742F41626C616765202000006A6198
:10694000202020202020202020206E65696E00005D
:106950002065696E6765736368616C746574212076
:106960000000206175736765736368616C7465749A
:10697000212000002D2D204D656EF52020202F3187
:1069800036202D2D00005452582D494420202043FC
:1069900054524C2D494400002045696E7374656C57
:1069A0006C756E67656E2020000077657264656E99
:1069B0002067656CEF7363687421000020204269D2
:1069C00074746520626569646520202000004B6E48
:1069D000EF706665206472F5636B656E21200000C0
:1069E00042697474652077617274656E202E2E2E54
:1069F0000000537065696368657262616E6B203177
:106A00002D34000020204E696368747320777572FE
:106A100064652020000020202067656CEF736368A8
:106A20007421202020200000204CEF736368756ED5
:106A300067206CE17566742000005175656C6C65AB
:106A4000202D2D2D3E205A69656C0000496E697419
:106A500069616C6973696572756E67210000205801
:106A60004D4F44454D20456D7066616E67200000B6
:106A700020584D4F44454D2053656E64756E672018
:106A80000000206A65747A74207374617274656E94
:106A9000212000004665686C65722D4E6575737423
:106AA000617274210000492E4F2E202D204E6575F5
:106AB0007374617274210000426974746520776197
:106AC0007274656E202E2E2E00002A2300002D2DBC
:106AD0002D3E204552524F522023313A202A2C205D
:106AE0004C46206665686C7400002D2D2D3E2045B7
:106AF00052524F522023323A202A2C204C462066F4
:106B000065686C7400002D2D2D3E204552524F5269
:106B10002042656665686C202A2D506F7369746920
:106B20006F6E203E204C462D506F736974696F6EF6
:106B300000002D2D2D3E204552524F5220425546E9
:106B40004645522D524F544154494F4E20535441C3
:106B50005254206E616368204C494E452D46454590
:106B600044002D2D2D3E204552524F52202A000028
:106B70002D2D2D3E204552524F52202300002D2D09
:106B80002D3E204552524F522042656665686C206A
:106B9000756E62656B616E6E74002D2D2D3E2052F8
:106BA0004F47455200002A50545452454C414953D6
:106BB0005F3023002A50545452454C4149535F31B1
:106BC00023002A414C4956455F30303023002A5477
:106BD000494546504153532300002A484F434850EB
:106BE0004153532300002A5350554C454E5F3132D8
:106BF000372300002A4B4F4E44454E5F3235352334
:106C000000002A4B4F50504C45525F414C542300DA
:106C10002A4B4F50504C45525F4E455523002A5247
:106C200045534554230025000707D007AB0DD80E68
:106C300081144A15571B201C7327A627AF360E3820
:106C40009346F8460752CA5339619E615F6D0474DA
:106C50004FC320CBFFFF00000707D007AB0DA00FED
:106C600081144A15571B841C7327A627AF360E388C
:106C70009346F8460752CA5339619E615F6D0474AA
:106C80004FC320CBFFFF000008070A070C070E07C1
:106C9000100712071407160718071A071C071E0704
:106CA000200722072407260728072A072C072E0774
:106CB000300732073407360738073A073C073E07E4
:106CC000400742074407460748074A074C074E0754
:106CD000500752075407560758075A075C075E07C4
:106CE000600762076407660768076A076C076E0734
:106CF000700772077407760778077A077C077E07A4
:106D0000800782078407860788078A078C078E0713
:106D1000900792079407960798079A079C079E0783
:106D2000A007A207A407A607A807AA07AC07AE07F3
:106D3000B007B207B407B607B807BA07BC07BE0763
:106D4000C007C207C407C607C807CA07CC07CE07D3
:106D5000D007AC0DB00DB40DB80DBC0DC00DC40DF9
:106D6000C80DCC0DD00DD40DD80DDC0DE00DE40D0B
:106D7000E80DEC0DF00DF40DF80DFC0D000E040EF9
:106D8000080E0C0E100E140E180E1C0E200E240EE3
:106D9000280E2C0E300E340E380E3C0E400E440ED3
:106DA000480E4C0E500E540E580E5C0E600E640EC3
:106DB000680E6C0E700E740E780E7C0E800E840EB3
:106DC000880E8C0E900E940E980E9C0EA00EA40EA3
:106DD000A80EAC0EB00EB40EB80EBC0EC00EC40E93
:106DE000C80ECC0ED00ED40ED80E821486148A147F
:106DF0008E14921496149A149E14A214A614AA1413
:106E0000AE14B214B614BA14BE14C214C614CA1402
:106E1000CE14D214D614DA14DE14E214E614EA14F2
:106E2000EE14F214F614FA14FE14021506150A15DF
:106E30000E15121516151A151E15221526152A15CA
:106E40002E15321536153A153E15421546154A15BA
:106E5000581B5C1B601B641B681B6C1B701B741B2A
:106E6000781B7C1B801B841B881B8C1B901B941B1A
:106E7000981B9C1BA01BA41BA81BAC1BB01BB41B0A
:106E8000B81BBC1BC01BC41BC81BCC1BD01BD41BFA
:106E9000D81BDC1BE01BE41BE81BEC1BF01BF41BEA
:106EA000F81BFC1B001C041C081C0C1C101C141CD4
:106EB000181C1C1C201C74277E27882792279C27BF
:106EC000A627B036BA36C436CE36D836E236EC36D9
:106ED000F63600370A3714371E37283732373C3733
:106EE000463750375A3764376E37783782378C37A2
:106EF0009637A037AA37B437BE37C837D237DC3712
:106F0000E637F037FA3704380E3894469E46A846DE
:106F1000B246BC46C646D046DA46E446EE46F84699
:106F2000085212521C52265230523A5244524E5279
:106F3000585262526C52765280528A5294529E52E9
:106F4000A852B252BC52C652D052DA52E452EE5259
:106F5000F85202530C53165320532A5334533E53C2
:106F6000485352535C53665370537A5384538E5331
:106F70009853A253AC53B653C053CA533A614461B9
:106F80004E61586162616C61766180618A61946171
:106F90009E61606D926DC46DF66D286E5A6E8C6E3A
:106FA000BE6EF06E226F546F866FB86FEA6F1C7002
:106FB0004E708070B270E470167148717A71AC7165
:106FC000DE71107242727472A672D8720A733C73C8
:106FD0006E73A073D273047450C382C3B4C3E6C388
:106FE00018C44AC47CC4AEC4E0C412C544C576C546
:106FF000A8C5DAC50CC63EC670C6A2C6D4C606C7AA
:1070000038C76AC79CC7CEC700C832C864C896C80C
:10701000C8C8FAC82CC95EC990C9C2C9F4C926CA71
:1070200058CA8ACABCCAEECA20CBFFFF08070A07A3
:107030000C070E07100712071407160718071A0780
:107040001C071E07200722072407260728072A07F0
:107050002C072E07300732073407360738073A0760
:107060003C073E07400742074407460748074A07D0
:107070004C074E07500752075407560758075A0740
:107080005C075E07600762076407660768076A07B0
:107090006C076E07700772077407760778077A0720
:1070A0007C077E07800782078407860788078A0790
:1070B0008C078E07900792079407960798079A0700
:1070C0009C079E07A007A207A407A607A807AA0770
:1070D000AC07AE07B007B207B407B607B807BA07E0
:1070E000BC07BE07C007C207C407C607C807CA0750
:1070F000CC07CE07D007AC0DB00DB40DB80DBC0D4C
:10710000C00DC40DC80DCC0DD00DD40DD80DDC0DA7
:10711000E00DE40DE80DEC0DF00DF40DF80DFC0D97
:10712000000E040E080E0C0E100E140E180E1C0E7F
:10713000200E240E280E2C0E300E340E380E3C0E6F
:10714000400E440E480E4C0E500E540E580E5C0E5F
:10715000600E640E680E6C0E700E740E780E7C0E4F
:10716000800E840E880E8C0E900E940E980E9C0E3F
:10717000A00EA40EA80EAC0EB00EB40EB80EBC0E2F
:10718000C00EC40EC80ECC0ED00ED40ED80EDC0E1F
:10719000E00EE40EE80EEC0EF00EF40EF80EFC0E0F
:1071A000000F040F080F0C0F100F140F180F1C0FF7
:1071B000200F240F280F2C0F300F340F380F3C0FE7
:1071C000400F440F480F4C0F500F540F580F5C0FD7
:1071D000600F640F680F6C0F700F740F780F7C0FC7
:1071E000800F840F880F8C0F900F940F980F9C0FB7
:1071F000A00F82148A1492149A14A214AA14B2141E
:10720000BA14C214CA14D214DA14E214EA14F2142E
:10721000FA1402150A1512151A1522152A15321517
:107220003A1542154A15581B601B681B701B781BCA
:10723000801B881B901B981BA01BA81BB01BB81B96
:10724000C01BC81BD01BD81BE01BE81BF01BF81B86
:10725000001C081C101C181C201C281C301C381C6E
:10726000401C481C501C581C601C681C701C781C5E
:10727000801C74277E27882792279C27A627B03654
:10728000BA36C436CE36D836E236EC36F636003765
:107290000A3714371E37283732373C3746375037CE
:1072A0005A3764376E37783782378C379637A0373E
:1072B000AA37B437BE37C837D237DC37E637F037AE
:1072C000FA3704380E3894469E46A846B246BC4665
:1072D000C646D046DA46E446EE46F8460852125212
:1072E0001C52265230523A5244524E525852625216
:1072F0006C52765280528A5294529E52A852B25286
:10730000BC52C652D052DA52E452EE52F8520253F4
:107310000C53165320532A5334533E53485352535D
:107320005C53665370537A5384538E539853A253CD
:10733000AC53B653C053CA533A6144614E6158616D
:1073400062616C61766180618A6194619E61606D49
:10735000926DC46DF66D286E5A6E8C6EBE6EF06EB8
:10736000226F546F866FB86FEA6F1C704E7080701A
:10737000B270E470167148717A71AC71DE7110727E
:1073800042727472A672D8720A733C736E73A073E1
:10739000D273047450C382C3B4C3E6C318C44AC4CE
:1073A0007CC4AEC4E0C412C544C576C5A8C5DAC560
:1073B0000CC63EC670C6A2C6D4C606C738C76AC7C2
:1073C0009CC7CEC700C832C864C896C8C8C8FAC827
:1073D0002CC95EC990C9C2C9F4C926CA58CA8ACA8A
:1073E000BCCAEECA20CBFFFFFA00F401E803D007C5
:1073F000A00F401F803E030006000C001900320061
:107400006400C800900101000200040008001000A0
:10741000200040008000644B323205230A2D0A22EE
:107420002800647D192505230A2D0A22280000075B
:107430000E091C1B1215383F363124232A2D707774
:107440007E796C6B6265484F464154535A5DE0E764
:10745000EEE9FCFBF2F5D8DFD6D1C4C3CACD9097D4
:107460009E998C8B8285A8AFA6A1B4B3BABDC7C0C4
:10747000C9CEDBDCD5D2FFF8F1F6E3E4EDEAB7B034
:10748000B9BEABACA5A28F88818693949D9A272024
:10749000292E3B3C35321F18111603040D0A575094
:1074A000595E4B4C45426F68616673747D7A898E74
:1074B000878095929B9CB1B6BFB8ADAAA3A4F9FEF4
:1074C000F7F0E5E2EBECC1C6CFC8DDDAD3D4696EE4
:1074D000676075727B7C51565F584D4A4344191E54
:1074E000171005020B0C21262F283D3A33344E4944
:1074F000404752555C5B7671787F6A6D64633E39B4
:10750000303722252C2B0601080F1A1D1413AEA9A3
:10751000A0A7B2B5BCBB9691989F8A8D8483DED913
:0E752000D0D7C2C5CCCBE6E1E8EFFAFDF4F31C
:00000001FF
